:020000040000FA
:1000000084EF5EF00000000000EF00F00000000050
:100010000000000000000000F3D7FFFF020E0D6E8D
:100020000D2EFED7000012008880FF0E996E889278
:10003000030E8714016E0150030A01E0F9D788828C
:1000400012000B6A0A6A096A00500402F4CF09F030
:10005000F3CF08F001500502F4CF0BF0F3CF0AF014
:1000600000500502F3500926F4500A22E86A0B22D8
:1000700001500402F3500926F4500A22E86A0B22C8
:1000800008C000F009C001F00AC002F00BC003F084
:100090001200086A096A100E0C6E0134083609361F
:1000A0000450085E0550D8A0053C095ED8B007D0C2
:1000B000045008260550D8B0053C0926D8900036D3
:1000C00001360C2EEAD71200AFDF996AA1CD87FF67
:1000D0008894A4DFA3DFA2DF888412008890996A45
:1000E000A1CD87FF88949ADF99DF98DF888412007A
:1000F0000301D8510D019B5D04E10301D7510D01AE
:100100009A5DD8B012000301DA510D019D5D04E142
:100110000301D9510D019C5DD8B01200800E9B19CE
:10012000006E800E005C02E1000E9A5DD8A0120005
:10013000800E9D19006E800E005C02E1000E9C5D39
:10014000D8A01200D3C304F0D4C305F09ACD00F0B8
:100150009BCD01F09EDF00C09FFD9CCD00F09DCDAA
:1001600001F0D5C304F0D6C305F06BDF9F51002624
:10017000000E01220301DF510024036EE051012033
:10018000046E04C000F0016A00C0A0FD03C0A1FD20
:10019000A5DFA0CDA1FDA2DF240E0D01A16F94DF8C
:1001A000F00E0D019E11A16FD3C304F0D4C305F06E
:1001B0009ACD00F09BCD01F06CDF08C000F009C0C3
:1001C00001F000500301D35D006E000600500D01E8
:1001D000A1137ADF12000D0187518B5D016E8851EA
:1001E0008C59026E01C092FD02C093FD8551895D5C
:1001F000946F86518A59956F800E0218006E800E9A
:10020000005C02E1000E015C0BE292510008926F6B
:100210009351000E9357FF0E986FFF0E996F04D005
:10022000010E986F000E996F800E9519006E800E6A
:10023000005C02E1000E945D0BE294510008946FA3
:100240009551000E9557FF0E966FFF0E976F04D0D5
:10025000010E966F000E976F9237929193379437F5
:100260009491953785CD9AFD86CD9BFD87CD9CFDDC
:1002700088CD9DFD8DCD9EFD3BDF800E0D01931938
:10028000006E800E9519005C02E19451925D42E28D
:1002900094CD00F095CD01F001320032019E01BCF9
:1002A000018E0050925D8E6F015093598F6F0D013A
:1002B00086518A1902E1895185192BE0800E8F1928
:1002C000006E800E005C02E1000E8E5D08E3985126
:1002D00087279951882394518E5F95518F5B965152
:1002E0008525006E97518621016E00C085FD01C0F5
:1002F00086FD92518E2793518F2300C09AFD01C035
:100300009BFD87CD9CFD88CD9DFD8DCD9EFDF0DEB6
:10031000CED742D092CD00F093CD01F00132003221
:10032000019E01BC018E00500D01945D906F015043
:100330009559916F0D0188518C1902E18B518719E4
:100340002BE0800E9119006E800E005C02E1000E21
:10035000905D08E396518527975186239251905FCF
:100360009351915B98518725006E99518821016EB8
:1003700000C087FD01C088FD9451902795519123BD
:1003800085CD9AFD86CD9BFD00C09CFD01C09DFDE5
:100390008DCD9EFDADDECED712007DCD00F0016A81
:1003A00000C07FFD7CCDA1FD99DE7FCDA1FD96DE55
:1003B0007ECDA1FD89DE1200800E0D018119006E37
:1003C000800E7D19005C02E17C51805D17E37CCDDD
:1003D00085FD7DCD86FD7ECD87FD7FCD88FD7CCDE5
:1003E00089FD7DCD8AFD82CD8BFD83CD8CFD84CDB5
:1003F0008DFDF1DE0D017C4B7D2BDED7120014DE6E
:10040000C50E0D01A16F60DEFF0E996E07DE8890AC
:100410008892888403DE02DE01DE87CF7CFD04DE65
:100420007CCD00F012000D015851545D016E01C0E9
:100430006DFD800E0118006E800E000A005C17E250
:100440006D510008036E046A000E6DBFFF0E045A62
:100450005CCD01F05DCD02F0013601900236025014
:10046000045C02E10150035CD8A0120012D05CCD04
:1004700001F05DCD02F0013601900236000E6DBF35
:10048000FF0E006E0250005C02E101506D5DD8A0CD
:1004900012005A51565D016E01C06DFD800E0118AB
:1004A000006E800E000A005C17E26D510008036EBA
:1004B000046A000E6DBFFF0E045A5CCD01F05DCDE5
:1004C00002F00136019002360250045C02E1015054
:1004D000035CD8A0120012D05CCD01F05DCD02F01B
:1004E000013601900236000E6DBFFF0E006E025005
:1004F000005C02E101506D5DD8A0120054CD7CFD7E
:1005000055CD7DFD5C5156257E6F5D5157217F6F26
:1005100058CD80FD59CD81FD5C515A5D826F5D5192
:100520005B59836F5ECD84FD47DF636B646B5C5109
:100530005625006E5D515721016E5C51585D046E69
:100540005D515959056E0450005C656F05500158A6
:10055000666F5C515425026E5D515521036E025049
:10056000005C676F03500158686F5C515A5D006E04
:100570005D515B59016E0250005C696F0350015878
:100580006A6F0450005C6B6F055001586C6F5CCD56
:1005900061FD5DCD62FD5CCD00F05DCD01F000360A
:1005A0000090013600C05FFD01C060FD00500308EF
:1005B0005F6F01C060FD000E6057010E6125016E86
:1005C000000E6221026E800E6419006E800E021809
:1005D000005C02E10150635DD8B0E7D05C51542566
:1005E000856F5D515521866F6351855F6451865BD0
:1005F0005C515A5D006E5D515B59016E6151002680
:100600006251012200C087FD01C088FD5C51585D28
:10061000896F5D5159598A6F6351892764518A23C3
:1006200000C08BFD01C08CFD5ECD8DFDD4DD0D01C4
:100630005C515425856F5D515521866F6351855FEF
:100640006451865B5C515625006E5D515721016EE9
:100650006151005E6251015A00C087FD01C088FDF2
:100660005C51585D896F5D5159598A6F6351892773
:1006700064518A2300C08BFD01C08CFD5ECD8DFDD1
:10068000AADD0D015C515A5D026E5D515B59036E2E
:1006900061510224856F62510320866F6B51855F23
:1006A0006C51865B63510224006E64510320016E1D
:1006B00000C087FD01C088FD6151025C896F6251F5
:1006C00003588A6F6951895F6A518A5B00C08BFD4C
:1006D00001C08CFD5ECD8DFD7EDD0D015C5156258A
:1006E000026E5D515721036E6151025C856F62514C
:1006F0000358866F6751855F6851865B6351025C62
:10070000006E64510358016E00C087FD01C088FD72
:1007100061510224896F625103208A6F6551895F9C
:1007200066518A5B00C08BFD01C08CFD5ECD8DFDE6
:1007300052DD800E0D016019006E800E005C02E13A
:10074000000E5F5D13E263CD00F064CD01F0003672
:1007500000900136003600900136060E0026000E8D
:10076000012200505F27015060231CD06151635D5E
:10077000036E62516459046E03C000F004C001F0BE
:100780000036009001360036009001360A0E002631
:10079000000E012200505F2701506023010E615FAF
:1007A000000E625B634B642B08D712000D01585199
:1007B000545D016E01C06DFD800E0118006E800E4B
:1007C000000A005C17E26D510008036E046A000E17
:1007D0006DBFFF0E045A5CCD01F05DCD02F0013615
:1007E000019002360250045C02E10150035CD8A083
:1007F000120012D05CCD01F05DCD02F00136019007
:100800000236000E6DBFFF0E006E0250005C02E16A
:1008100001506D5DD8A012005A51565D016E01C0A5
:100820006DFD800E0118006E800E000A005C17E25C
:100830006D510008036E046A000E6DBFFF0E045A6E
:100840005CCD01F05DCD02F0013601900236025020
:10085000045C02E10150035CD8A0120012D05CCD10
:1008600001F05DCD02F0013601900236000E6DBF41
:10087000FF0E006E0250005C02E101506D5DD8A0D9
:1008800012005C515425856F5D515521866F56CD00
:1008900087FD57CD88FD5C51585D896F5D51595971
:1008A0008A6F56CD8BFD57CD8CFD5ECD8DFD93DCD3
:1008B0000D015C515425856F5D515521866F5ACDD0
:1008C00087FD5BCD88FD5C51585D896F5D5159593D
:1008D0008A6F5ACD8BFD5BCD8CFD5ECD8DFD7BDCB3
:1008E00054CD85FD55CD86FD0D015C515625876F94
:1008F0005D515721886F54CD89FD55CD8AFD5C51DE
:100900005A5D8B6F5D515B598C6F5ECD8DFD63DCE5
:1009100058CD85FD59CD86FD0D015C515625876F5B
:100920005D515721886F58CD89FD59CD8AFD5C51A5
:100930005A5D8B6F5D515B598C6F5ECD8DFD4BDCCD
:100940000D01636B646B5C515625006E5D51572140
:10095000016E5C51585D046E5D515959056E04502D
:10096000005C656F05500158666F5C515425026E3E
:100970005D515521036E0250005C676F03500158B2
:10098000686F5C515A5D006E5D515B59016E02509B
:10099000005C696F035001586A6F0450005C6B6F14
:1009A000055001586C6F5CCD61FD5DCD62FD5CCD85
:1009B00000F05DCD01F000360090013600C05FFD13
:1009C00001C060FD005003085F6F01C060FD000EB4
:1009D0006057010E6125016E000E6221026E800ECD
:1009E0006419006E800E0218005C02E10150635D24
:1009F000D8B00BD15C5154259A6F5D5155219B6F36
:100A000063519A5F64519B5B5C515A5D9C6F5D5171
:100A10005B599D6F61519C2762519D235ECD9EFD68
:100A200078EC00F00D015C51585D9A6F5D51595999
:100A30009B6F63519A2764519B235C515A5D9C6F55
:100A40005D515B599D6F61519C2762519D235ECD25
:100A50009EFD78EC00F00D015C5154259A6F5D51BC
:100A600055219B6F63519A5F64519B5B5C51562586
:100A70009C6F5D5157219D6F61519C5F62519D5BE1
:100A80005ECD9EFD78EC00F00D015C51585D9A6FD3
:100A90005D5159599B6F63519A2764519B235C5157
:100AA00056259C6F5D5157219D6F61519C5F62512E
:100AB0009D5B5ECD9EFD78EC00F00D015C515A5DB2
:100AC000006E5D515B59016E615100249A6F625155
:100AD00001209B6F6B519A5F6C519B5B63510024AB
:100AE0009C6F645101209D6F5ECD9EFD78EC00F0FF
:100AF0000D015C515A5D006E5D515B59016E615193
:100B0000005C9A6F625101589B6F69519A5F6A51FC
:100B10009B5B635100249C6F645101209D6F5ECDEF
:100B20009EFD78EC00F00D015C515625006E5D5184
:100B30005721016E6151005C9A6F625101589B6FA1
:100B400067519A5F68519B5B6351005C9C6F645175
:100B500001589D6F5ECD9EFD78EC00F00D015C515B
:100B60005625006E5D515721016E615100249A6F28
:100B7000625101209B6F65519A5F66519B5B635187
:100B8000005C9C6F645101589D6F5ECD9EFD78ECBA
:100B900000F0800E0D016019006E800E005C02E115
:100BA000000E5F5D13E263CD00F064CD01F000360E
:100BB00000900136003600900136060E0026000E29
:100BC000012200505F27015060231CD06151635DFA
:100BD000036E62516459046E03C000F004C001F05A
:100BE0000036009001360036009001360A0E0026CD
:100BF000000E012200505F2701506023010E615F4B
:100C0000000E625B634B642BE4D6120058CDA1FD4D
:100C100064EC00F057CD00F0000E016ED5C304F077
:100C2000D6C305F021EC00F00D01565100247C6F75
:100C3000000E01207D6F0301E1510D017C270301AE
:100C4000E2510D017D23240E7E6FCDEC01F054CDD9
:100C5000E9FF55CDEAFFEE5211E054CDE9FF55CD45
:100C6000EAFF200EEE5C0D01A16F6EEC00F0544B1C
:100C7000552BC00EA16F64EC00F0E9D7120054CDE3
:100C800085FD55CD86FD56CD87FD57CD88FD58CDC8
:100C900089FD59CD8AFD56CD8BFD57CD8CFD5CCDA0
:100CA0008DFDEBEC00F058CD85FD59CD86FD56CD80
:100CB00087FD57CD88FD58CD89FD59CD8AFD5ACD88
:100CC0008BFD5BCD8CFD5CCD8DFDEBEC00F058CD4C
:100CD00085FD59CD86FD5ACD87FD5BCD88FD54CD70
:100CE00089FD55CD8AFD5ACD8BFD5BCD8CFD5CCD4C
:100CF0008DFDEBEC00F054CD85FD55CD86FD5ACD34
:100D000087FD5BCD88FD54CD89FD55CD8AFD56CD3F
:100D10008BFD57CD8CFD5CCD8DFDEBEC00F0120012
:100D20000D01736B746B716B726B0301D8510D0104
:100D3000555D04E10301D7510D01545D17E2030134
:100D4000DA510D01575D04E10301D9510D01565DE2
:100D50000DE2000E591902E1000E581907E0000ECD
:100D60005B1902E1000E5A1901E001D0120058513E
:100D70005425016E59515521026E02500301D85D70
:100D800002E10150D75D0BE20D0154510301D75D23
:100D90000D01586F55510301D8590D01596F0D01BF
:100DA0005A515625016E5B515721026E02500301C4
:100DB000DA5D02E10150D95D0BE20D0156510301EC
:100DC000D95D0D015A6F57510301DA590D015B6F5F
:100DD0000D01D3C304F0D4C305F054CD00F055CDBC
:100DE00001F049EC00F008C000F009C001F000C0BB
:100DF00075FD585154257A6F595155217B6FD3C3D6
:100E000004F0D4C305F07ACD00F07BCD01F049ECBD
:100E100000F008C000F009C001F000C076FDD3C3A7
:100E200004F0D4C305F054CD00F055CD01F049ECE9
:100E300000F000C06BFD01C06CFD010E7A5D006E1C
:100E4000000E7B59016ED3C304F0D4C305F049EC06
:100E500000F000C06DFD01C06EFDD3C304F0D4C32B
:100E600005F05CCD00F05DCD01F049EC00F008C06C
:100E700000F009C001F0000E026E0150025C02E1B8
:100E80000050000811E2D3C304F0D4C305F05CCDD8
:100E900000F05DCD01F049EC00F0010E00246F6F11
:100EA000000E0120706F0ED0D3C304F0D4C305F040
:100EB0005CCD00F05DCD01F049EC00F000C06FFDAD
:100EC00001C070FD696B6A6B656B666B5B51665D3B
:100ED00002E15A51655DD8B008D1736B716B726BCA
:100EE0006BCD67FD6CCD68FD68516E5D02E16751A9
:100EF0006D5DD8A0F3D0D3C304F0D4C305F054CDB6
:100F000000F055CD01F049EC00F067510024636F0B
:100F100068510120646F6B51635F6C51645B655174
:100F20005625006E66515721016ED5C304F0D6C315
:100F300005F021EC00F0635100247C6F6451012026
:100F40007D6F0301DF510D017C270301E0510D018D
:100F50007D23240E7E6FCDEC01F014EC00F00D012A
:100F60005F51665D02E15E51655D07E27051725D41
:100F700002E16F51715D01E202D0746B14D07151C6
:100F80006925006E72516A21016E00506025F66E6F
:100F900001506121F76E000E6221F86E0900F5CF55
:100FA00074FD714B722B755100081CE275CD00F079
:100FB00074CD77FD005004E07733779FFF0FFBD7A8
:100FC00075510301D35D006E00C001F073CD00F0D8
:100FD000015004E000360090FF0FFBD700500D01D8
:100FE000771302D074CD77FD68516C1902E16B5113
:100FF00067191BE17551000818E2FFEC01F000C011
:1010000078FD0D0175510301D35D016E01C002F041
:10101000FF0E016E025004E001360190FF0FFBD776
:101020000150001600500D01771368516E1902E14E
:101030006D51671945E17651000842E2FFEC01F07D
:1010400000C078FD0D0176510301D35D006E00C034
:1010500001F0FF0E006E015004E000360090FF0F1B
:10106000FBD700500D017717000E0301D41902E1E0
:10107000080ED3190FE176CD01F0FF0E006E01507E
:1010800004E00032009EFF0FFBD700500D017815E1
:10109000796F14D00D01020E7625006E016A000EE4
:1010A000012200C001F0FF0E006E015004E000328A
:1010B000009EFF0FFBD700507815796F7951771399
:1010C00077CDA1FD6EEC00F0C40EA16F64EC00F0D2
:1010D00074CD73FD0D01674B682B06D76F516927DF
:1010E00070516A23654B662BF1D612000C0E0D0170
:1010F0005225E96E000E5321EA6EEE50010A1CE102
:10110000040E5225E16E000E5321E26E060E5225AA
:10111000E96E000E5321EA6EEECFE6FF050E522572
:10112000E16E000E5321E26E070E5225E96E000EAD
:101130005321EA6EEECFE6FF020E5225E96E000E55
:101140005321EA6EEECF54FD000E556F000E556F21
:10115000030E5225E96E000E5321EA6EEECF56FDC6
:10116000000E576F000E576F040E5225E96E000EE9
:101170005321EA6EEECF58FD000E596F000E596FE5
:10118000050E5225E96E000E5321EA6EEECF5AFD90
:10119000000E5B6F000E5B6F060E5225E96E000EAF
:1011A0005321EA6EEECF5CFD000E5D6F000E5D6FA9
:1011B000070E5225E96E000E5321EA6EEECF5EFD5A
:1011C000000E5F6F000E5F6F080E5225E96E000E75
:1011D0005321EA6EEECF60FDEECF61FDEECF62FDF2
:1011E0009FDD1200060E0D015225E96E000E5321FF
:1011F000EA6EEECF54FDEECF55FD020E5225E96E9C
:10120000000E5321EA6EEECF01F001C056FD5633B9
:10121000569F5633569F5633569F030E5225E96EFE
:10122000000E5321EA6EEECF01F001C057FD573397
:10123000579F5733579F5733579F810E586FE6DCA0
:101240001200020E0D015225E96E000E5321EA6EC6
:10125000EECF01F001C054FD000E556F030E522574
:10126000E96E000E5321EA6EEECF00F000C056FD8D
:10127000000E576F040E5225D96E000E5321DA6E00
:10128000DE500124586F596B000E5923010E585F30
:10129000000E595B050E5225D96E000E5321DA6EF1
:1012A000DE5000245A6F5B6B000E5B23010E5A5F09
:1012B000000E5B5B080E5C6FE2DC1200020E0D019B
:1012C0005225E96E000E5321EA6EEECF01F001C007
:1012D00054FD000E556F030E5225E96E000E53218A
:1012E000EA6EEECF00F000C056FD000E576F040E00
:1012F0005225D96E000E5321DA6EDE500124586F4C
:10130000596B000E5923010E585F000E595B050EF4
:101310005225D96E000E5321DA6EDE5000245A6F2A
:101320005B6B000E5B23010E5A5F000E5B5B070ECA
:101330005225E96E000E5321EA6EEECF5CFD000EE1
:101340005D6F000E5D6F080E5E6F13EC02F0040E11
:101350005225E96E000E5321EA6E050EEE5C54E351
:10136000050E5225E96E000E5321EA6E050EEE5C65
:101370004BE3020E5225E96E000E5321EA6EEECFCA
:1013800001F00150010F546F556B000E5523030EF1
:101390005225E96E000E5321EA6EEECF00F00050A8
:1013A000010F566F576B000E5723040E5225D96E4E
:1013B000000E5321DA6EDE500124586F596B000E77
:1013C0005923020E585F000E595B050E5225D96E47
:1013D000000E5321DA6EDE5000245A6F5B6B000E54
:1013E0005B23020E5A5F000E5B5B070E5225E96E0F
:1013F000000E5321EA6EEECF5CFD000E5D6F000E15
:101400005D6F5E6BD6EC03F0080E5225E96E000EA0
:101410005321EA6EEECF54FDEECF55FD020E52255C
:10142000E96E000E5321EA6E060E5225D96E000EAB
:101430005321DA6EDECF05F00550EE24006E016A0E
:10144000000E0122020E0024036E000E0120046E25
:10145000030E026E03C000F004C001F0025007E06A
:1014600001320032019E01BC018EFF0FF8D700C08F
:1014700056FD030E5225E96E000E5321EA6E05500B
:10148000EE24006E016A000E0122020E0024036E9B
:10149000000E0120046E030E026E03C000F004C0B3
:1014A00001F0025007E001320032019E01BC018EC2
:1014B000FF0FF8D700C057FD810E586F06EC06F0FD
:1014C0001200020E0D015225E96E000E5321EA6E44
:1014D000EECF01F001C07CFD000E7D6F030E5225A2
:1014E000E96E000E5321EA6EEECF00F000C07EFDE3
:1014F000000E7F6F040E5225D96E000E5321DA6E56
:10150000DE500124806F816B000E8123010E805F0D
:10151000000E815B050E5225D96E000E5321DA6E46
:10152000DE500024826F836B000E8323010E825FE6
:10153000000E835B080E846FDCEC01F0040E522574
:10154000E96E000E5321EA6E050EEE5C48E3050ECF
:101550005225E96E000E5321EA6E050EEE5C3FE364
:10156000020E5225E96E000E5321EA6EEECF01F015
:101570000150010F546F556B000E5523030E522579
:10158000E96E000E5321EA6EEECF00F00050010F1D
:10159000566F576B000E5723040E5225D96E000E5E
:1015A0005321DA6EDE500124586F596B000E592317
:1015B000020E585F000E595B050E5225D96E000EC3
:1015C0005321DA6EDE5000245A6F5B6B000E5B23F2
:1015D000020E5A5F000E5B5B5C6B3FEC06F0070E81
:1015E0000D015225E96E000E5321EA6EEECF54FD37
:1015F000EECF55FD020E5225E96E000E5321EA6E24
:10160000060E5225D96E000E5321DA6EDECF05F09C
:101610000550EE24006E016A000E0122020E002425
:10162000036E000E0120046E030E026E03C000F074
:1016300004C001F0025007E001320032019E01BCFB
:10164000018EFF0FF8D70D0100C056FD030E522585
:10165000E96E000E5321EA6E0550EE24006E016A19
:10166000000E0122020E0024036E000E0120046E03
:10167000030E026E03C000F004C001F0025007E048
:1016800001320032019E01BC018EFF0FF8D70D011F
:1016900000C057FD810E586F06EC06F012000D01D8
:1016A0004B6B4C6B100E0601D725D96E000ED8215E
:1016B000DA6EDECF01F0DECF02F002500D014C5D9C
:1016C00002E101504B5D32E2120E0601D725E96EB0
:1016D000000ED821EA6EEECF03F0EECF04F04BCD32
:1016E00000F04CCD01F0003600900136005003248C
:1016F000E96E01500420EA6EEECF00F0EECF01F06B
:1017000000C04DFD01C04EFD060E0024E96E000E26
:101710000120EA6EEE50010A05E14DCD52FD4ECD9D
:1017200053FD8FDD0D014B4B4C2BBCD712004BCD25
:1017300002F04CCD03F002C000F003C001F0024AF9
:10174000032A00C0E9FF01C0EAFFEE5201E0F3D72F
:101750000D014B51025C006E4C510358016E010E9D
:10176000005E000E015A12000D014B6B4C6BD7C688
:10177000E9FFD8C6EAFFEECF01F0EECF02F002504B
:101780004C5D02E101504B5D32E2020E0601D725AD
:10179000E96E000ED821EA6EEECF03F0EECF04F032
:1017A0004BCD00F04CCD01F00036009001360050DA
:1017B0000324E96E01500420EA6EEECF00F0EECF74
:1017C00001F000C04DFD01C04EFD0F0E0024E96E7A
:1017D000000E0120EA6EEE50010A05E14DCD52FDEA
:1017E0004ECD53FDFFDC0D014B4B4C2BC0D71200EF
:1017F0000D014B515A0804E3410E4B5DD8B04B8BA1
:101800004BCD00F012000D014B6B4C6B040E06012A
:10181000D725D96E000ED821DA6EDECF01F0DECFEB
:1018200002F002500D014C5D02E101504B5D32E2CD
:10183000060E0601D725E96E000ED821EA6EEECF1E
:1018400003F0EECF04F04BCD00F04CCD01F00036AC
:101850000090013600500324E96E01500420EA6E26
:10186000EECF00F0EECF01F000C04DFD01C04EFD07
:101870000B0E0024E96E000E0120EA6EEE50010A04
:1018800005E14DCD52FD4ECD53FD30DC0D014B4BEE
:101890004C2BBCD712000D014B6B4C6B0C0E060190
:1018A000D725D96E000ED821DA6EDECF01F0DECF5B
:1018B00002F002500D014C5D02E101504B5D32E23D
:1018C0000E0E0601D725E96E000ED821EA6EEECF86
:1018D00003F0EECF04F04BCD00F04CCD01F000361C
:1018E0000090013600500324E96E01500420EA6E96
:1018F000EECF00F0EECF01F000C04DFD01C04EFD77
:10190000110E0024E96E000E0120EA6EEE50010A6D
:1019100005E14DCD52FD4ECD53FDD0DC0D014B4BBD
:101920004C2BBCD712000D014B6B4C6B080E060103
:10193000D725D96E000ED821DA6EDECF01F0DECFCA
:1019400002F002500D014C5D02E101504B5D32E2AC
:101950000A0E0601D725E96E000ED821EA6EEECFF9
:1019600003F0EECF04F04BCD00F04CCD01F000368B
:101970000090013600500324E96E01500420EA6E05
:10198000EECF00F0EECF01F000C04DFD01C04EFDE6
:10199000100E0024E96E000E0120EA6EEE50010ADE
:1019A00005E14DCD52FD4ECD53FD8BDD0D014B4B71
:1019B0004C2BBCD712000D01506B516B14EC00F096
:1019C0000D014C510301DF250D017C6F4D510301C9
:1019D000E0210D017D6F240E7E6FCDEC01F0B00E85
:1019E0000D01A16F64EC00F08890996A0D014F51D0
:1019F000515D02E14E51505D0DE24BCD87FF889461
:101A00000EEC00F00EEC00F00EEC00F08884504B71
:101A1000512BECD7B20EA16F64EC00F012004BCD4D
:101A200004F04CCD05F004C002F005C003F0044AF8
:101A3000052A4DCD00F04ECD01F00D014D4B4E2B42
:101A400000C0E9FF01C0EAFF02C0E1FF03C0E2FFFE
:101A5000EECFE6FF02C0E9FF03C0EAFFEE5201E06D
:101A6000E2D74BCD00F04CCD01F012003A0E0D6ED6
:101A70000D2EFED7000012004BCD04F04CCD05F02A
:101A800004C0E9FF05C0EAFFEE5203E0044A052A5C
:101A9000F7D704C002F005C003F0044A052A4DCD73
:101AA00000F04ECD01F00D014D4B4E2B00C0E9FF73
:101AB00001C0EAFF02C0E1FF03C0E2FFEECFE6FF94
:101AC00002C0E9FF03C0EAFFEE5201E0E2D74BCDCE
:101AD00000F04CCD01F01200829486808292BB0E01
:101AE0000D01546F020E556F0A0E566F060E576F9A
:101AF000810E586F06EC06F0120082948690828266
:101B0000060E0D01546F030E556F0A0E566F060E2A
:101B1000576F810E586F06EC06F01200200E0D0173
:101B2000496F4A6B0301E4B305D047CD4BFD60DE3E
:101B300000C047FD0D01120E4B6F030E4C6FF7DD19
:101B400000C048FD150E005C19E3200E4B6F000E1F
:101B50004C6F580E4D6F030E4E6F61DF120E4B6FC0
:101B6000030E4C6F6F0E4D6F030E4E6F58DFEE0E6F
:101B7000526F0C0E536FF2EC08F012000301E4A157
:101B800020D00D01485100081BE24805006E016A93
:101B9000000E015A120E0024E16E030E0120E26EC7
:101BA000E66A200E4B6F000E4C6F7F0E4D6F030EDA
:101BB0004E6F35DFEE0E526F0C0E536FF2EC08F0E5
:101BC0000CD047CD49FD120E0D014B6F030E4C6F2B
:101BD000490E4D6F0D0E4E6F4FDF0D01200E4B6FF6
:101BE000000E4C6F120E4D6F030E4E6F18DFEE0E8F
:101BF000526F0C0E536FF2EC08F012008294869034
:101C00008292B00E0D01546F020E556F0A0E566F80
:101C1000060E576F810E586F06EC06F01200C30EC9
:101C2000C21647CD00F000360090003600900050FC
:101C3000C2121CDFC282C2A201D0FDD7C4CF01F004
:101C4000006AC3500012000E011212000D014B6B0E
:101C50004C6B4D6BD5C64EFDD6C64FFDACDE0D01AF
:101C60004B6BD5C64CFDD6C64DFDD9C64EFDDAC66A
:101C70004FFDA1DE47CDD7F648CDD8F6C4DD53DE03
:101C80000ADE0DDD71DD1200828486808292920E62
:101C90000D01546F020E556F0A0E566F060E576FE8
:101CA000810E586F06EC06F01200829486808282C4
:101CB0009F0E0D01546F020E556F0A0E566F060EE1
:101CC000576F810E586F06EC06F0120082848690E2
:101CD0008292C70E0D01546F020E556F0A0E566F99
:101CE000060E576F810E586F06EC06F012008284C4
:101CF00086908282D60E0D01546F020E556F0A0E29
:101D0000566F060E576F810E586F06EC06F01200E4
:101D1000490E0D01476F02DF1200550E0D01476F8E
:101D2000FDDE1200120E0D014B6F030E4C6F960E6E
:101D30004D6F030E4E6F73DE0301E491E493350E95
:101D40000D014B6F000E4C6F710E4D6F030E4E6FF9
:101D500066DECA0E476F040E486F78DF12004F0E22
:101D60000D01476FDBDE1200530E0D01476FD6DE0B
:101D700012006B0E0D01476F0C0E486F67DF1200EB
:101D8000500E0D01476FCADE1200520E0D01476F53
:101D9000C5DE1200450E0D01476FC0DE1200570E62
:101DA0000D01476FBBDE1200540E0D01476FB6DE0A
:101DB0001200120E0D014B6F030E4C6F050E4D6F8E
:101DC000030E4E6F2CDE0301E491200E0D014B6FCC
:101DD000000E4C6F700E4D6F030E4E6F20DEDF0E47
:101DE000476F060E486F32DF1200510E0D01476F2C
:101DF00095DE1200590E0D01476F90DE12004B0E5A
:101E00000D01476F8BDE1200827282A20BD0F50E9D
:101E10000D014B6F000E4C6F010E4D6F030E4E6F98
:101E2000FEDD0CD082B20AD00D01F50E4B6F000E14
:101E30004C6FF50E4D6F020E4E6FF1DD660E526F58
:101E4000090E536FF2EC08F01200867086A00BD0DA
:101E5000400E0D014B6F010E4C6F280E4D6F030E9F
:101E60004E6FDDDD0CD086B00AD00D01400E4B6FF9
:101E7000010E4C6F2C0E4D6F030E4E6FD0DDDE0E3B
:101E8000526F090E536FF2EC08F01200827482A4B4
:101E90000BD03C0E0D014B6F010E4C6F480E4D6F79
:101EA000030E4E6FBCDD0CD082B40AD00D013C0E87
:101EB0004B6F010E4C6FED0E4D6F020E4E6FAFDD8E
:101EC000867086A00AD0400E4B6F010E4C6FF10E4B
:101ED0004D6F020E4E6FA3DD0BD086B009D0400EC1
:101EE0004B6F010E4C6FE50E4D6F020E4E6F97DD7E
:101EF000827282A20AD0F50E4B6F000E4C6FE90E73
:101F00004D6F020E4E6F8BDD0BD082B209D0F50EF5
:101F10004B6F000E4C6FFD0E4D6F020E4E6F7FDD4E
:101F2000640E526F0A0E536FF2EC08F0DE0E0D01D4
:101F3000526F090E536FF2EC08F0660E0D01526FEE
:101F4000090E536FF2EC08F0120082948690829290
:101F50003C0E0D014B6F010E4C6FF90E4D6F020ED2
:101F60004E6F5DDD400E4B6F010E4C6FE10E4D6FFD
:101F7000020E4E6F54DDF50E4B6F000E4C6FAC0E23
:101F80004D6F020E4E6F4BDD640E526F0A0E536F93
:101F9000F2EC08F0DE0E0D01526F090E536FF2ECF9
:101FA00008F0660E0D01526F090E536FF2EC08F047
:101FB00012005A0E0D01476F080E486F47DE1200DF
:101FC0000301E473E4A30BD0350E0D014B6F000E3B
:101FD0004C6F300E4D6F030E4E6F21DD0DD003019F
:101FE000E4B30AD0350E0D014B6F000E4C6F3A0E64
:101FF0004D6F030E4E6F13DD0D01320E526F0C0E3E
:10200000536F5EEC09F01200827482A40BD03C0E78
:102010000D014B6F010E4C6F7B0E4D6F030E4E6F1B
:10202000FEDC0CD082B40AD00D013C0E4B6F010EC9
:102030004C6F540E4D6F030E4E6FF1DC640E526FF9
:102040000A0E536FF2EC08F01200DF0E0D01476F1D
:10205000060E486FFBDD12008284868082823C0E71
:102060000D014B6F010E4C6F4C0E4D6F030E4E6FFA
:10207000D6DC400E4B6F010E4C6F500E4D6F030EB1
:102080004E6FCDDCF50E4B6F000E4C6F440E4D6F56
:10209000030E4E6FC4DC640E526F0A0E536FF2ECE7
:1020A00008F0DE0E0D01526F090E536FF2EC08F0CE
:1020B000660E0D01526F090E536FF2EC08F012001C
:1020C000340E0C6EF10E0D6E0D2EFED70C2EFCD7BD
:1020D000000000001200F250026EF29E0500FF6A3E
:1020E0000150FE6E0050FD6E02BEF28E1200050E13
:1020F0000B6E0F0E0C6EF10E0D6E0D2EFED70C2E0C
:10210000FCD70B2EFAD71200060E0C6E2B0E0D6E9E
:102110000D2EFED70C2EFCD71200F40E0D01476FCA
:10212000070E486F93DD12000301AE6BDF0E0D0149
:10213000476F060E486F8ADD12000450085E055096
:10214000D8A0053C095E0650D8A0063C0A5E0750A0
:10215000D8A0073C0B5E0336070E0C6E033408361E
:1021600009360A360B36045003A00ED0085E05501F
:10217000D8A0053C095E0650D8A0063C0A5E075070
:10218000D8A0073C0B5E0DD008260550D8B0053C02
:1021900009260650D8B0063C0A260750D8B0073C9E
:1021A0000B2603360C2EDAD70234083609360A36E7
:1021B0000B36045003A00ED0085E0550D8A0053C95
:1021C000095E0650D8A0063C0A5E0750D8A0073C1E
:1021D0000B5E0DD008260550D8B0053C09260650E8
:1021E000D8B0063C0A260750D8B0073C0B2602366A
:1021F000070E0C6E0234083609360A360B360450C8
:1022000002A00ED0085E0550D8A0053C095E06501D
:10221000D8A0063C0A5E0750D8A0073C0B5E0DD044
:1022200008260550D8B0053C09260650D8B0063C13
:102230000A260750D8B0073C0B2602360C2EDAD7F8
:102240000134083609360A360B36045002A00ED087
:10225000085E0550D8A0053C095E0650D8A0063C93
:102260000A5E0750D8A0073C0B5E0DD0082605502B
:10227000D8B0053C09260650D8B0063C0A260750BF
:10228000D8B0073C0B260136070E0C6E0134083619
:1022900009360A360B36045001A00ED0085E0550F0
:1022A000D8A0053C095E0650D8A0063C0A5E07503F
:1022B000D8A0073C0B5E0DD008260550D8B0053CD1
:1022C00009260650D8B0063C0A260750D8B0073C6D
:1022D0000B2601360C2EDAD70034083609360A36BA
:1022E0000B36045001A00ED0085E0550D8A0053C66
:1022F000095E0650D8A0063C0A5E0750D8A0073CED
:102300000B5E0DD008260550D8B0053C09260650B6
:10231000D8B0063C0A260750D8B0073C0B2600363A
:10232000070E0C6E0034083609360A360B36045098
:1023300000A00ED0085E0550D8A0053C095E0650EE
:10234000D8A0063C0A5E0750D8A0073C0B5E0DD013
:1023500008260550D8B0053C09260650D8B0063CE2
:102360000A260750D8B0073C0B2600360C2EDAD7C9
:1023700000B00ED0045008260550D8B0053C092600
:102380000650D8B0063C0A260750D8B0073C0B26AA
:1023900012000B1E0A1E091E081E082AD8B4092A9C
:1023A000D8B40A2AD8B40B2A1200480E0D01476F80
:1023B0008EEC0DF01200470E0D01476F8EEC0DF004
:1023C00012005A0E0D01476F8EEC0DF012004C0EEC
:1023D0000D01476F8EEC0DF01200440E0D01476F9A
:1023E0008EEC0DF01200A80E0D01476F090E486F1C
:1023F0002DDC050E0B6E0F0E0C6EF10E0D6E0D2EFC
:10240000FED70C2EFCD70B2EFAD7FEEC0DF0290EC2
:102410000B6E960E0C6E7F0E0D6E0D2EFED70C2ED3
:10242000FCD70B2EFAD730DC290E0B6E960E0C6EF5
:102430007F0E0D6E0D2EFED70C2EFCD70B2EFAD76D
:1024400056DC290E0B6E960E0C6E7F0E0D6E0D2E49
:10245000FED70C2EFCD70B2EFAD738DC290E0B6ECC
:10246000960E0C6E7F0E0D6E0D2EFED70C2EFCD729
:102470000B2EFAD71ADC290E0B6E960E0C6E7F0E01
:102480000D6E0D2EFED70C2EFCD70B2EFAD76CEC52
:102490000DF0290E0B6E960E0C6E7F0E0D6E0D2E2E
:1024A000FED70C2EFCD70B2EFAD77DEC0DF0290EA3
:1024B0000B6E960E0C6E7F0E0D6E0D2EFED70C2E33
:1024C000FCD70B2EFAD7829486908292010E0301DC
:1024D000AE6FA80E0D01476F090E486F26EC0EF087
:1024E0001200460E0D01476F8EEC0DF01200410EEA
:1024F0000D01476F8EEC0DF012004A0E0D01476F73
:102500008EEC0DF012004D0E0D01476F8EEC0DF0AC
:1025100012004E0E0D01476F8EEC0DF01200200ED2
:102520000D01476F8EEC0DF012000301E4810D01E7
:10253000476B8EEC0DF00301E4911200430E0D0188
:10254000476F8EEC0DF01200580E0D01476F8EECA8
:102550000DF01200420E0D01476F8EEC0DF01200CF
:10256000560E0D01476F8EEC0DF012008984899A8A
:10257000000E0301DE1902E1800EDD1908E1000EF4
:10258000D21902E1400ED11902E1BEDD01D098DD81
:10259000C1C3E1FFC2C3E2FFC7C3E6FFBFC300F090
:1025A000C0C301F098DD12003FCDD7F340CDD8F382
:1025B00041CDD9F3000E0301DA6F42CDD3F3000E03
:1025C000D46FD3C304F0D4C305F03FCD00F040CDA9
:1025D00001F049EC00F000C0D5F301C0D6F3D9C337
:1025E00004F0DAC305F021EC00F000C0D5F601C01C
:1025F000D6F6D9C300F0DAC301F001320032019EF1
:1026000001320032019E01320032019ED5C304F036
:10261000D6C305F021EC00F000C0D9F601C0DAF60F
:102620009A949A929A909A988884888288808888C6
:10263000FF0E996E88985BDD888859DD810E0D014B
:10264000A16F64EC00F042CD04F0000E056ED7C31C
:1026500000F0D8C301F049EC00F000C07CFD01C0DF
:102660007DFD430E0D017E6FCDEC01F0D5C37CFDE9
:10267000D6C37DFD410E0D017E6FCDEC01F006014C
:10268000D951D5250D014E6F0601DA51D6210D0124
:102690004F6F0301DF6BE06BD5C6E1F3D6C6E2F303
:1026A0000D014B6B4C6B4D6BDBEC0CF0900E030192
:1026B000E36F0D017C6B7D6B420E7E6FCDEC01F004
:1026C000D5C67CFDD6C67DFD400E0D017E6FCDECDE
:1026D00001F012001E0E0301BF6F1C0EC06F470EEB
:1026E000C16F0D0EC26FC26A070EC012C08EC280CB
:1026F00012003FCDDBF340CDDCF312009294929AAE
:10270000840E0301DB6F030EDC6F3FCDDDF340CDA4
:10271000DEF341CDD1F342CDD2F343CDC7F344CD67
:10272000C8F3C36BC46BC56BC66B1200000E0D0102
:10273000405D02E143513F5D2DE345514325006E6D
:10274000016A000E0122010E005C026E000E0158AB
:10275000036E4051035C02E13F51025C1BE3000E3B
:10276000425D02E14451415D15E346514425006E4E
:10277000016A000E0122010E005C026E000E01587B
:10278000036E4251035C02E14151025C03E3010E1E
:10279000006E1200006A1200220E0C6E086A096AAE
:1027A0000A6A0B6A0C06D8B41FD0D8900B320A32D2
:1027B000093208320332023201320032D8A0F2D795
:1027C0000C06D8B409D0045008260550092206503A
:1027D0000A2207500B22EAD7045008260550092286
:1027E00006500A2207500B2212008994898A000E93
:1027F0000301DE1902E1800EDD1908E1000ED21995
:1028000002E1400ED11902E17FDC01D059DCC1C3E5
:10281000E1FFC2C3E2FFC8C3E6FFBFC300F0C0C30D
:1028200001F059DC12000450000A12E10550000AC0
:102830000FE10650000A0CE10750000A09E1FF0E03
:10284000006EFF0E016EFF0E026E7F0E036E120011
:102850000C6A07BE0C2A0D6A0B6A0A6A096A086AC2
:102860000350021001100010D8B484D00350071890
:102870000E6E0EBE0D1E07AE0BD0041E051E061EEC
:10288000071E042AD8B4052AD8B4062AD8B4072AC1
:1028900003AE0BD0001E011E021E031E002AD8B478
:1028A000012AD8B4022AD8B4032A035007100E6EA6
:1028B0000EBE1CD042DC0CBE36D00DAE5BD0001E6E
:1028C000011E021E031E002AD8B4012AD8B4022A0F
:1028D000D8B4032A081E091E0A1E0B1E082AD8B4E3
:1028E000092AD8B40A2AD8B40B2A44D007AE15D086
:1028F00003BE0DD003500B6E02500A6E0150096EDC
:102900000050086E036A026A016A006AD6D7036A39
:10291000026A016A006A002A000C031E021E011EE0
:10292000001E0C8EC7D7082AD8B4092AD8B40A2AA0
:10293000D8B40B2A0450085CD8A4BFD70550095C52
:10294000D8A4BBD706500A5CD8A4B7D707500B5CF5
:10295000D8A4B3D70B6A0A6A096A086A002AD8B4ED
:10296000012AD8B4022AD8B4032A03AEA6D70E6A25
:102970000E88FF0C0E6A0CA001D00BDD000F1200B8
:102980000D01336B346B080E0601D725D96E000E8E
:10299000D821DA6EDECF01F0DECF02F002500D0159
:1029A000345D02E10150335DD8B07CD00A0E0601DF
:1029B000D725E96E000ED821EA6EEECF03F0EECFF8
:1029C00004F033CD00F034CD01F000360090013634
:1029D00000500324E96E01500420EA6EEECF00F0AF
:1029E000EECF01F000C035FD01C036FD2FCD3FFD1B
:1029F00030CD40FD31CD41FD32CD42FD020E0024EF
:102A0000E96E000E0120EA6EEECF43FD030E0024B6
:102A1000E96E000E0120EA6EEECF44FD040E0024A4
:102A2000E96E000E0120EA6EEECF45FD050E002492
:102A3000E96E000E0120EA6EEECF46FD77DE005013
:102A4000010A2CE11D0E3525E96E000E3621EA6ED5
:102A5000EECF01F0EECF02F0EECF03F0EECF04F0B8
:102A6000000E006E041808E10050031805E1005044
:102A7000021802E10150000A11E01D0E3525E96E31
:102A8000000E3621EA6EEECF00F0EECF01F0EECF71
:102A900002F0EECF03F06BEC10F012000D01334B9F
:102AA000342B71D7336B346B0C0E0601D725D96EDE
:102AB000000ED821DA6EDECF01F0DECF02F0025038
:102AC0000D01345D02E10150335DD8B07CD00E0EB3
:102AD0000601D725E96E000ED821EA6EEECF03F08D
:102AE000EECF04F033CD00F034CD01F0003600908D
:102AF000013600500324E96E01500420EA6EEECF47
:102B000000F0EECF01F000C037FD01C038FD2FCD41
:102B10003FFD30CD40FD31CD41FD32CD42FD020EB5
:102B20000024E96E000E0120EA6EEECF43FD030E95
:102B30000024E96E000E0120EA6EEECF44FD040E83
:102B40000024E96E000E0120EA6EEECF45FD050E71
:102B50000024E96E000E0120EA6EEECF46FDE6DDB0
:102B60000050010A2CE11E0E3725E96E000E3821B7
:102B7000EA6EEECF01F0EECF02F0EECF03F0EECF33
:102B800004F0000E006E041808E10050031805E17F
:102B90000050021802E10150000A11E01E0E372514
:102BA000E96E000E3821EA6EEECF00F0EECF01F0B4
:102BB000EECF02F0EECF03F06BEC10F012000D013F
:102BC000334B342B71D7336B346BD7C6E9FFD8C680
:102BD000EAFFEECF01F0EECF02F00250345D02E1E9
:102BE0000150335DD8B07CD0020E0601D725E96EC6
:102BF000000ED821EA6EEECF03F0EECF04F033CD15
:102C000000F034CD01F0003600900136005003246E
:102C1000E96E01500420EA6EEECF00F0EECF01F035
:102C200000C039FD01C03AFD2FCD3FFD30CD40FD44
:102C300031CD41FD32CD42FD020E0024E96E000E81
:102C40000120EA6EEECF43FD030E0024E96E000E74
:102C50000120EA6EEECF44FD040E0024E96E000E62
:102C60000120EA6EEECF45FD050E0024E96E000E50
:102C70000120EA6EEECF46FD59DD0050010A2CE13D
:102C80001C0E3925E96E000E3A21EA6EEECF01F0F6
:102C9000EECF02F0EECF03F0EECF04F0000E006EA8
:102CA000041808E10050031805E10050021802E181
:102CB0000150000A11E01C0E3925E96E000E3A2180
:102CC000EA6EEECF00F0EECF01F0EECF02F0EECFE5
:102CD00003F06BEC10F012000D01334B342B75D761
:102CE000336B346B040E0601D725D96E000ED82144
:102CF000DA6EDECF01F0DECF02F002500D01345D5E
:102D000002E10150335DD8B07CD0060E0601D72514
:102D1000E96E000ED821EA6EEECF03F0EECF04F09C
:102D200033CD00F034CD01F0003600900136005074
:102D30000324E96E01500420EA6EEECF00F0EECFDE
:102D400001F000C03BFD01C03CFD2FCD3FFD30CD6B
:102D500040FD31CD41FD32CD42FD020E0024E96E31
:102D6000000E0120EA6EEECF43FD030E0024E96E53
:102D7000000E0120EA6EEECF44FD040E0024E96E41
:102D8000000E0120EA6EEECF45FD050E0024E96E2F
:102D9000000E0120EA6EEECF46FDC8DC0050010AAD
:102DA0002CE1190E3B25E96E000E3C21EA6EEECFB8
:102DB00001F0EECF02F0EECF03F0EECF04F0000E04
:102DC000006E041808E10050031805E100500218D5
:102DD00002E10150000A11E0190E3B25E96E000ED8
:102DE0003C21EA6EEECF00F0EECF01F0EECF02F024
:102DF000EECF03F06BEC10F012000D01334B342BCF
:102E000071D7336B346B100E0601D725D96E000EC7
:102E1000D821DA6EDECF01F0DECF02F002500D01D4
:102E2000345D02E10150335DD8B07CD0120E060152
:102E3000D725E96E000ED821EA6EEECF03F0EECF73
:102E400004F033CD00F034CD01F0003600900136AF
:102E500000500324E96E01500420EA6EEECF00F02A
:102E6000EECF01F000C03DFD01C03EFD2FCD3FFD86
:102E700030CD40FD31CD41FD32CD42FD020E00246A
:102E8000E96E000E0120EA6EEECF43FD030E002432
:102E9000E96E000E0120EA6EEECF44FD040E002420
:102EA000E96E000E0120EA6EEECF45FD050E00240E
:102EB000E96E000E0120EA6EEECF46FD37DC0050D1
:102EC000010A2CE1130E3D25E96E000E3E21EA6E4B
:102ED000EECF01F0EECF02F0EECF03F0EECF04F034
:102EE000000E006E041808E10050031805E10050C0
:102EF000021802E10150000A11E0130E3D25E96EAF
:102F0000000E3E21EA6EEECF00F0EECF01F0EECFE4
:102F100002F0EECF03F06BEC10F012000D01334B1A
:102F2000342B71D712000D0EC16E6AEC13F09A9615
:102F300088969A9A889A9A9C889C9494949298904D
:102F4000829482928690F00E0D013F6F000E406FCA
:102F5000800E416F080E426FD4EC12F00301E3873C
:102F6000E3C3A1FD64EC00F00301E385E3C3A1FD2D
:102F700064EC00F00301E393E3C3A1FD64EC00F013
:102F8000F00E0D013F6F000E406F800E416F000E7E
:102F9000426F436B010E446F7EEC13F0840E0D0103
:102FA0003F6F030E406F79EC13F00301976B986B42
:102FB000996B12000D01336B346B080E0601D72597
:102FC000D96E000ED821DA6EDECF01F0DECF02F02E
:102FD00002500D01345D02E10150335DD8B0B5D02F
:102FE0000A0E0601D725E96E000ED821EA6EEECF53
:102FF00003F0EECF04F033CD00F034CD01F0003615
:103000000090013600500324E96E01500420EA6E5E
:10301000EECF00F0EECF01F000C035FD01C036FD6F
:103020002FCD3FFD30CD40FD31CD41FD32CD42FDB4
:10303000020E0024E96E000E0120EA6EEECF43FD81
:10304000030E0024E96E000E0120EA6EEECF44FD6F
:10305000040E0024E96E000E0120EA6EEECF45FD5D
:10306000050E0024E96E000E0120EA6EEECF46FD4B
:1030700096EC13F00050010A65E1110E3525E96E5A
:10308000000E3621EA6EEECF01F0EECF02F0EECF69
:1030900003F0EECF04F0000E006E041808E10050BB
:1030A000031805E10050021802E10150000A10E087
:1030B000110E3525E96E000E3621EA6EEECF00F0D6
:1030C000EECF01F0EECF02F0EECF03F06BEC10F09C
:1030D000030199510D01361903E135510301981986
:1030E0002DE1190E0D013525E96E000E3621EA6E2F
:1030F000EECF01F0EECF02F0EECF03F0EECF04F012
:10310000000E006E041808E10050031805E100509D
:10311000021802E10150000A11E00D01190E3525D7
:10312000E96E000E3621EA6EEECF00F0EECF01F030
:10313000EECF02F0EECF03F06BEC10F00301986BD2
:10314000996B1200334B342B38D7336B346B0C0E26
:103150000601D725D96E000ED821DA6EDECF01F038
:10316000DECF02F002500D01345D02E10150335D0B
:10317000D8B0B5D00E0E0601D725E96E000ED821C5
:10318000EA6EEECF03F0EECF04F033CD00F034CD95
:1031900001F000360090013600500324E96E015022
:1031A0000420EA6EEECF00F0EECF01F000C037FD54
:1031B00001C038FD2FCD3FFD30CD40FD31CD41FD6B
:1031C00032CD42FD020E0024E96E000E0120EA6EAF
:1031D000EECF43FD030E0024E96E000E0120EA6EDF
:1031E000EECF44FD040E0024E96E000E0120EA6ECD
:1031F000EECF45FD050E0024E96E000E0120EA6EBB
:10320000EECF46FD96EC13F00050010A65E1120E78
:103210003725E96E000E3821EA6EEECF01F0EECFD1
:1032200002F0EECF03F0EECF04F0000E006E0418B3
:1032300008E10050031805E10050021802E10150B6
:10324000000A10E0120E3725E96E000E3821EA6EF2
:10325000EECF00F0EECF01F0EECF02F0EECF03F0B4
:103260006BEC10F0030199510D01381903E137514E
:10327000030198192DE11A0E0D013725E96E000E94
:103280003821EA6EEECF01F0EECF02F0EECF03F080
:10329000EECF04F0000E006E041808E10050031891
:1032A00005E10050021802E10150000A11E00D0191
:1032B0001A0E3725E96E000E3821EA6EEECF00F0C7
:1032C000EECF01F0EECF02F0EECF03F06BEC10F09A
:1032D0000301986B996B1200334B342B38D7336B47
:1032E000346BD7C6E9FFD8C6EAFFEECF01F0EECFC8
:1032F00002F00250345D02E10150335DD8B0B5D028
:10330000020E0601D725E96E000ED821EA6EEECF37
:1033100003F0EECF04F033CD00F034CD01F00036F1
:103320000090013600500324E96E01500420EA6E3B
:10333000EECF00F0EECF01F000C039FD01C03AFD44
:103340002FCD3FFD30CD40FD31CD41FD32CD42FD91
:10335000020E0024E96E000E0120EA6EEECF43FD5E
:10336000030E0024E96E000E0120EA6EEECF44FD4C
:10337000040E0024E96E000E0120EA6EEECF45FD3A
:10338000050E0024E96E000E0120EA6EEECF46FD28
:1033900096EC13F00050010A65E1100E3925E96E34
:1033A000000E3A21EA6EEECF01F0EECF02F0EECF42
:1033B00003F0EECF04F0000E006E041808E1005098
:1033C000031805E10050021802E10150000A10E064
:1033D000100E3925E96E000E3A21EA6EEECF00F0AC
:1033E000EECF01F0EECF02F0EECF03F06BEC10F079
:1033F000030199510D013A1903E13951030198195B
:103400002DE1180E0D013925E96E000E3A21EA6E04
:10341000EECF01F0EECF02F0EECF03F0EECF04F0EE
:10342000000E006E041808E10050031805E100507A
:10343000021802E10150000A11E00D01180E3925B1
:10344000E96E000E3A21EA6EEECF00F0EECF01F009
:10345000EECF02F0EECF03F06BEC10F00301986BAF
:10346000996B1200334B342B3CD7336B346B040E07
:103470000601D725D96E000ED821DA6EDECF01F015
:10348000DECF02F002500D01345D02E10150335DE8
:10349000D8B0B5D0060E0601D725E96E000ED821AA
:1034A000EA6EEECF03F0EECF04F033CD00F034CD72
:1034B00001F000360090013600500324E96E0150FF
:1034C0000420EA6EEECF00F0EECF01F000C03BFD2D
:1034D00001C03CFD2FCD3FFD30CD40FD31CD41FD44
:1034E00032CD42FD020E0024E96E000E0120EA6E8C
:1034F000EECF43FD030E0024E96E000E0120EA6EBC
:10350000EECF44FD040E0024E96E000E0120EA6EA9
:10351000EECF45FD050E0024E96E000E0120EA6E97
:10352000EECF46FD96EC13F00050010A65E10D0E5A
:103530003B25E96E000E3C21EA6EEECF01F0EECFA6
:1035400002F0EECF03F0EECF04F0000E006E041890
:1035500008E10050031805E10050021802E1015093
:10356000000A10E00D0E3B25E96E000E3C21EA6ECC
:10357000EECF00F0EECF01F0EECF02F0EECF03F091
:103580006BEC10F0030199510D013C1903E13B5123
:10359000030198192DE1150E0D013B25E96E000E72
:1035A0003C21EA6EEECF01F0EECF02F0EECF03F059
:1035B000EECF04F0000E006E041808E1005003186E
:1035C00005E10050021802E10150000A11E00D016E
:1035D000150E3B25E96E000E3C21EA6EEECF00F0A1
:1035E000EECF01F0EECF02F0EECF03F06BEC10F077
:1035F0000301986B996B1200334B342B38D7336B24
:10360000346B100E0601D725D96E000ED821DA6E64
:10361000DECF01F0DECF02F002500D01345D02E199
:103620000150335DD8B0B5D0120E0601D725E96E32
:10363000000ED821EA6EEECF03F0EECF04F033CDCA
:1036400000F034CD01F00036009001360050032424
:10365000E96E01500420EA6EEECF00F0EECF01F0EB
:1036600000C03DFD01C03EFD2FCD3FFD30CD40FDF2
:1036700031CD41FD32CD42FD020E0024E96E000E37
:103680000120EA6EEECF43FD030E0024E96E000E2A
:103690000120EA6EEECF44FD040E0024E96E000E18
:1036A0000120EA6EEECF45FD050E0024E96E000E06
:1036B0000120EA6EEECF46FD96EC13F00050010AB1
:1036C00065E1070E3D25E96E000E3E21EA6EEECF64
:1036D00001F0EECF02F0EECF03F0EECF04F0000EDB
:1036E000006E041808E10050031805E100500218AC
:1036F00002E10150000A10E0070E3D25E96E000EC0
:103700003E21EA6EEECF00F0EECF01F0EECF02F0F8
:10371000EECF03F06BEC10F0030199510D013E194F
:1037200003E13D51030198192DE10F0E0D013D25D7
:10373000E96E000E3E21EA6EEECF01F0EECF02F010
:10374000EECF03F0EECF04F0000E006E041808E197
:103750000050031805E10050021802E10150000A70
:1037600011E00D010F0E3D25E96E000E3E21EA6EBF
:10377000EECF00F0EECF01F0EECF02F0EECF03F08F
:103780006BEC10F00301986B996B1200334B342BE8
:1037900038D70301986B996B12000D01336B346BB2
:1037A000080E0601D725D96E000ED821DA6EDECFBD
:1037B00001F0DECF02F002500D01345D02E1015054
:1037C000335DD8B081D00A0E0601D725E96E000E10
:1037D000D821EA6EEECF03F0EECF04F033CD00F047
:1037E00034CD01F000360090013600500324E96E1C
:1037F00001500420EA6EEECF00F0EECF01F000C0E1
:1038000035FD01C036FD2FCD3FFD30CD40FD31CD22
:1038100041FD32CD42FD020E0024E96E000E012072
:10382000EA6EEECF43FD030E0024E96E000E012088
:10383000EA6EEECF44FD040E0024E96E000E012076
:10384000EA6EEECF45FD050E0024E96E000E012064
:10385000EA6EEECF46FD96EC13F00050010A30E11F
:1038600035CD98F336CD99F3150E3525E96E000E5A
:103870003621EA6EEECF01F0EECF02F0EECF03F08C
:10388000EECF04F0000E006E041808E1005003189B
:1038900005E10050021802E10150000A11E0150E86
:1038A0003525E96E000E3621EA6EEECF00F0EECF40
:1038B00001F0EECF02F0EECF03F06BEC10F012004F
:1038C0000D01334B342B6CD7336B346B0C0E06016C
:1038D000D725D96E000ED821DA6EDECF01F0DECF0B
:1038E00002F002500D01345D02E10150335DD8B0A9
:1038F00081D00E0E0601D725E96E000ED821EA6EA2
:10390000EECF03F0EECF04F033CD00F034CD01F074
:1039100000360090013600500324E96E0150042067
:10392000EA6EEECF00F0EECF01F000C037FD01C02F
:1039300038FD2FCD3FFD30CD40FD31CD41FD32CDA5
:1039400042FD020E0024E96E000E0120EA6EEECF69
:1039500043FD030E0024E96E000E0120EA6EEECF57
:1039600044FD040E0024E96E000E0120EA6EEECF45
:1039700045FD050E0024E96E000E0120EA6EEECF33
:1039800046FD96EC13F00050010A30E137CD98F374
:1039900038CD99F3160E3725E96E000E3821EA6E00
:1039A000EECF01F0EECF02F0EECF03F0EECF04F059
:1039B000000E006E041808E10050031805E10050E5
:1039C000021802E10150000A11E0160E3725E96ED7
:1039D000000E3821EA6EEECF00F0EECF01F0EECF10
:1039E00002F0EECF03F06BEC10F012000D01334B40
:1039F000342B6CD7336B346BD7C6E9FFD8C6EAFFDC
:103A0000EECF01F0EECF02F00250345D02E1015042
:103A1000335DD8B081D0020E0601D725E96E000EC5
:103A2000D821EA6EEECF03F0EECF04F033CD00F0F4
:103A300034CD01F000360090013600500324E96EC9
:103A400001500420EA6EEECF00F0EECF01F000C08E
:103A500039FD01C03AFD2FCD3FFD30CD40FD31CDC8
:103A600041FD32CD42FD020E0024E96E000E012020
:103A7000EA6EEECF43FD030E0024E96E000E012036
:103A8000EA6EEECF44FD040E0024E96E000E012024
:103A9000EA6EEECF45FD050E0024E96E000E012012
:103AA000EA6EEECF46FD96EC13F00050010A30E1CD
:103AB00039CD98F33ACD99F3140E3925E96E000EFD
:103AC0003A21EA6EEECF01F0EECF02F0EECF03F036
:103AD000EECF04F0000E006E041808E10050031849
:103AE00005E10050021802E10150000A11E0140E35
:103AF0003925E96E000E3A21EA6EEECF00F0EECFE6
:103B000001F0EECF02F0EECF03F06BEC10F01200FC
:103B10000D01334B342B70D7336B346B040E06011D
:103B2000D725D96E000ED821DA6EDECF01F0DECFB8
:103B300002F002500D01345D02E10150335DD8B056
:103B400081D0060E0601D725E96E000ED821EA6E57
:103B5000EECF03F0EECF04F033CD00F034CD01F022
:103B600000360090013600500324E96E0150042015
:103B7000EA6EEECF00F0EECF01F000C03BFD01C0D9
:103B80003CFD2FCD3FFD30CD40FD31CD41FD32CD4F
:103B900042FD020E0024E96E000E0120EA6EEECF17
:103BA00043FD030E0024E96E000E0120EA6EEECF05
:103BB00044FD040E0024E96E000E0120EA6EEECFF3
:103BC00045FD050E0024E96E000E0120EA6EEECFE1
:103BD00046FD96EC13F00050010A30E13BCD98F31E
:103BE0003CCD99F3110E3B25E96E000E3C21EA6EA7
:103BF000EECF01F0EECF02F0EECF03F0EECF04F007
:103C0000000E006E041808E10050031805E1005092
:103C1000021802E10150000A11E0110E3B25E96E85
:103C2000000E3C21EA6EEECF00F0EECF01F0EECFB9
:103C300002F0EECF03F06BEC10F012000D01334BED
:103C4000342B6CD7336B346B100E0601D725D96E2D
:103C5000000ED821DA6EDECF01F0DECF02F0025086
:103C60000D01345D02E10150335DD8B081D0120EF8
:103C70000601D725E96E000ED821EA6EEECF03F0DB
:103C8000EECF04F033CD00F034CD01F000360090DB
:103C9000013600500324E96E01500420EA6EEECF95
:103CA00000F0EECF01F000C03DFD01C03EFD2FCD84
:103CB0003FFD30CD40FD31CD41FD32CD42FD020E04
:103CC0000024E96E000E0120EA6EEECF43FD030EE4
:103CD0000024E96E000E0120EA6EEECF44FD040ED2
:103CE0000024E96E000E0120EA6EEECF45FD050EC0
:103CF0000024E96E000E0120EA6EEECF46FD96EC40
:103D000013F00050010A30E13DCD98F33ECD99F318
:103D10000B0E3D25E96E000E3E21EA6EEECF01F05E
:103D2000EECF02F0EECF03F0EECF04F0000E006E07
:103D3000041808E10050031805E10050021802E1E0
:103D40000150000A11E00B0E3D25E96E000E3E21E8
:103D5000EA6EEECF00F0EECF01F0EECF02F0EECF44
:103D600003F06BEC10F012000D01334B342B6CD7C9
:103D700012002FCDCDF330CDCEF331CDC9F332CDFE
:103D8000CAF333CDCFF334CDD0F335CDCBF336CD2D
:103D9000CCF312008994899A84EC10F0C1C3E1FF3E
:103DA000C2C3E2FFC8C3E6FFBFC300F0C0C301F057
:103DB0006BEC10F001500301DC5D02E10050DB5DB3
:103DC000010ED8B0000E0D012F6F84EC10F0C1C3AE
:103DD000E1FFC2C3E2FFC8C3E6FFBFC300F0C0C338
:103DE00001F06BEC10F001500301DC5D02E10050CA
:103DF000DB5D010ED8B0000E026E02500D012F15D2
:103E0000006E00C02FFD1200B6EC12F00301CD5180
:103E1000005C0D01336F0301CE5101580D01346F69
:103E2000F5EC13F00301CF51005C0D01356F030178
:103E3000D05101580D01366F33CD00F034CD01F073
:103E4000000E34BFFF0E026E036EDDC304F0DEC34E
:103E500005F0000E066E076ECCEC13F00301CD5199
:103E6000C95D046ECE51CA59056E000E066E076E0E
:103E700013EC14F000C033FD01C034FD35CD00F06B
:103E800036CD01F0000E0D0136BFFF0E026E036E3F
:103E9000D1C304F0D2C305F0000E066E076ECCEC61
:103EA00013F00301CF51CB5D046ED051CC59056E98
:103EB000000E066E076E13EC14F000500301D15D86
:103EC0000D01356F01500301D2590D01366F800E7F
:103ED0003419006E800E005C02E1000E335D0BE3CE
:103EE0000301DE510D01345D04E10301DD510D01DB
:103EF000335D01E203D0010E006E1200800E361910
:103F0000006E800E005C02E1000E355D0BE30301E4
:103F1000D2510D01365D04E10301D1510D01355D32
:103F200001E203D0010E006E12000301C3510D0126
:103F3000335D016E0301C4510D013459026E01C09D
:103F400037FD02C038FD0301C5510D01355D396FE4
:103F50000301C6510D0136593A6F33CDC3F334CD49
:103F6000C4F335CDC5F336CDC6F3800E000A006E1E
:103F7000800E0218005C02E1015005081DE3800E6E
:103F8000000A006E800E3A19005C02E13951050802
:103F900013E3800E3819006E7F0E005C02E1FB0E09
:103FA000375D0AE3800E3A19006E7F0E005C02E175
:103FB000FB0E395D01E303D0010E006E12002FCD20
:103FC000E1FF30CDE2FF33CDE6FF34CDE6FF31CD6A
:103FD000E1FF32CDE2FF35CDE6FF36CDE6FF006AE8
:103FE0001200020E0601DF6F000EE06FDB0EE16FC4
:103FF000060EE26F010EE36F000EE46FD30EE56F65
:10400000060EE66FE76BE86B030EEB6F000EEC6FCE
:10401000690EED6F060EEE6FEF6BF06B490EDB6F06
:10402000060EDC6F6F0EDD6F060EDE6FB10E696F70
:10403000060E6A6F8F0E6B6F060E6C6FD70ED36F06
:10404000070ED46FB50E6D6F070E6E6F080E070169
:10405000F46F000EF56F0A0EF66F080EF76FF86B2F
:10406000F96BFC6BFD6B010E0801006F000E016F18
:10407000080E026F080E036F046B056B930E086F3A
:10408000070E096F130E0A6F070E0B6FF30E0C6FFE
:10409000060E0D6F330E0E6F070E0F6F730E106F3F
:1040A000070E116F530E126F070E136F880E146FE9
:1040B000040E156F680E166F040E176FA80E186F9A
:1040C000040E196F010E0401CA6F000ECB6FC80EEB
:1040D000CC6F040ECD6F010ECE6F000ECF6F660E4B
:1040E000D06F040ED16F1B0ED26F000ED36FEB0E8C
:1040F000D46F030ED56F020ED66F000ED76FE70E8A
:10410000D86F030ED96F010EDA6F000EDB6F210E30
:10411000DC6F040EDD6F440E0301E76F040EE86FE1
:10412000230EEB6F040EEC6FC50EED6F050EEE6FF8
:10413000A40EEF6F050EF06FE60EF16F050EF26F35
:10414000280EF36F060EF46F070EF56F060EF66F6E
:10415000830EF76F050EF86FFF0EF96F040EFA6FFE
:10416000DE0EFB6F040EFC6F200EFD6F050EFE6F62
:10417000620EFF6F050E0401006F410E016F050E08
:10418000026F8D0E036F0B0E046F6C0E056F0B0E1E
:10419000066FAE0E076F0B0E086FF00E096F0B0E59
:1041A0000A6FCF0E0B6F0B0E0C6F4B0E0D6F0B0EBD
:1041B0000E6FC70E0F6F0A0E106FA60E116F0A0E4C
:1041C000126FE80E136F0A0E146F2A0E156F0B0E86
:1041D000166F090E176F0B0E186F110E196F0C0E5C
:1041E0001A6FB00E1B6F0C0E1C6F8F0E1D6F0C0E16
:1041F0001E6FD10E666F0C0E676F0E0E1F6F0D0EC9
:10420000206FEE0EC86F0C0EC96F540E216F0C0E8E
:10421000226F320E0301E96F0C0EEA6F070E0C01DC
:104220006B6F000E6C6F810E6D6F0C0E6E6F6F6B8F
:10423000706B736B746B010E776F000E786F7F0E6F
:10424000796F0C0E7A6F7B6B7C6BC20E7F6F080EE2
:10425000806FA20E816F080E826FE40E836F080ECE
:10426000846F240E856F090E866F040E876F090E0A
:10427000886F820E896F080E8A6F3A0E8B6F080E58
:104280008C6F1A0E8D6F080E8E6F030E08015A6F19
:10429000000E5B6F7C0E5C6F080E5D6F5E6B5F6B7C
:1042A000626B636B070E666F000E676F6E0E686F52
:1042B000080E696F6A6B6B6B200E6E6F0A0E6F6F64
:1042C000FE0E706F090E716F420E726F0A0E736FE1
:1042D000840E746F0A0E756F640E7C6F0A0E7D6F0C
:1042E000DE0E7E6F090E7F6F660E806F090E816F86
:1042F000440E766F090E776F860E786F090E796F10
:10430000BC0E7A6F090E7B6F0901A86BA96BAC6BB1
:10431000AD6B010EB06F000EB16FE50EB26F030E04
:10432000B36FB46BB56BB86BB96B9E0E0301E56FE1
:10433000030EE66FDF0E0601496F060E4A6F4B6BE8
:10434000100E4C6F900E4D6F080E4E6F1B0E4F6F80
:10435000020E506F516B526B536B070E546F070E6A
:10436000556F200E566F020E576F010E586F596B26
:104370005A6B5B6B5C6B5D6B5E6B5F6B606B616BF9
:10438000626B636B646B656B666B676B686BDF0E90
:104390006F6F060E706F716B200E726F980E736FD9
:1043A000080E746FF60E756F010E766F776B786B73
:1043B000796B070E7A6F070E7B6F200E7C6F020EF3
:1043C0007D6F010E7E6F7F6B806B816B826B836B69
:1043D000846B856B866B876B886B896B8A6B8B6B49
:1043E0008C6B8D6B8E6BDF0EB16F060EB26F030E92
:1043F000B36F3B0EB46F8A0EB56F120EB66F030E1D
:10440000B76F040EB86F0A0EB96F020EBA6FBB6BAE
:10441000BC6BBD6B070EBE6F070EBF6F200EC06F6B
:10442000020EC16F010EC26FC36BC46BC56BC66B4E
:10443000C76BC86BC96BCA6B1A0ECB6F210ECC6FE2
:10444000000ECD6F000ECE6FCF6BD06BD16BD26BE9
:10445000DF0E8F6F060E906F030E916F530E926FEB
:104460008A0E936F120E946F030E956F040E966F63
:104470004E0E976F020E986F996B9A6B9B6B070E9F
:104480009C6F070E9D6F200E9E6F020E9F6F010E98
:10449000A06FA16BA26BA36BA46BA56BA66BA76BA4
:1044A000A86B720EA96F1D0EAA6F000EAB6F000EE7
:1044B000AC6FAD6BAE6BAF6BB06BDF0E0701D76F40
:1044C000060ED86FB10ED96F060EDA6F370EDB6F9E
:1044D000360EDC6F370EDD6F360EDE6F000EDF6FCF
:1044E000610EE06F000EE16F010EE26FE36BE46BB3
:1044F000E56BE66BE76BE86BE96BEA6BEB6BEC6B20
:10450000ED6BEE6BEF6BF06BF16BF26BF36BDF0E41
:10451000B56F060EB66F030EB76F6B0EB86F8A0ECF
:10452000B96F120EBA6F030EBB6F040EBC6F5F0E35
:10453000BD6F020EBE6FBF6BC06BC16B070EC26F4B
:10454000070EC36F200EC46F020EC56F010EC66F3B
:10455000C76BC86BC96BCA6BCB6BCC6BCD6BCE6BAF
:10456000E60ECF6F230ED06F000ED16F000ED26F0C
:10457000D36BD46BD56BD66BF40E936F070E946F21
:10458000BB0E956F630E966F2A0E976F120E986F83
:10459000030E996F040E9A6F2E0E9B6F020E9C6F86
:1045A0009D6B9E6B9F6B070EA06F070EA16F200E79
:1045B000A26F020EA36F010EA46FA56BA66BA76B73
:1045C000A86BA96BAA6BAB6BAC6B240EAD6F1D0E09
:1045D000AE6F000EAF6F000EB06FB16BB26BB36B0E
:1045E000B46BF40E136F070E146F080E156F180ED0
:1045F000166FD00E176F080E186F330E196F020E5C
:104600001A6F1B6B1C6B1D6B070E1E6F070E1F6F47
:10461000200E206F020E216F010E226F236B246B80
:10462000256B266B276B286B296B2A6B2B6B2C6BEE
:104630002D6B2E6B2F6B306B316B326BF40E0601D2
:10464000F36F070EF46F080EF56F200EF66FD00EA5
:10465000F76F080EF86FDB0EF96F010EFA6FFB6B48
:10466000FC6BFD6B070EFE6F070EFF6F200E070140
:10467000006F020E016F010E026F036B046B056B7E
:10468000066B076B086B096B0A6B0B6B0C6B0D6B86
:104690000E6B0F6B106B116B126BF40E336F070EFA
:1046A000346F080E356F280E366FD80E376F080E30
:1046B000386F8A0E396F010E3A6F3B6B3C6B3D6B66
:1046C000070E3E6F070E3F6F200E406F020E416FC8
:1046D000010E426F436B446B456B466B476B486BF7
:1046E000496B4A6B4B6B4C6B4D6B4E6B4F6B506B0E
:1046F000516B526BF40E736F070E746F080E756F6B
:10470000300E766FA00E776F080E786FA60E796F59
:10471000010E7A6F7B6B7C6B7D6B070E7E6F070ED5
:104720007F6F200E806F020E816F010E826F836B90
:10473000846B856B866B876B886B896B8A6B8B6BE5
:104740008C6B8D6B8E6B8F6B906B916B926BF40E91
:10475000536F070E546F080E556F380E566FE00EEC
:10476000576F080E586F500E596F010E5A6F5B6BE2
:104770005C6B5D6B070E5E6F070E5F6F200E606FE8
:10478000020E616F010E626F636B646B656B666B2B
:10479000676B686B696B6A6B6B6B6C6B6D6B6E6B6D
:1047A0006F6B706B716B726BF40E0401886F070E88
:1047B000896F080E8A6F400E8B6FE00E8C6F080EAB
:1047C0008D6F6D0E8E6F010E8F6F906B916B926B74
:1047D000070E936F070E946F200E956F020E966F63
:1047E000010E976F986B996B9A6B9B6B9C6B9D6B93
:1047F0009E6B9F6BA06BA16BA26BA36BA46BA56B55
:10480000A66BA76BF40E686F070E696F080E6A6FD0
:10481000480E6B6F900E6C6F080E6D6FC20E6E6F50
:10482000010E6F6F706B716B726B070E736F070EFB
:10483000746F200E756F020E766F010E776F786BB6
:10484000796B7A6B7B6B7C6B7D6B7E6B7F6B806B2C
:10485000816B826B836B846B856B866B876BF40ECD
:10486000A86F070EA96F580EAA6F080EAB6F280E1F
:10487000AC6F080EAD6FD50EAE6F010EAF6FB06BA3
:10488000B16BB26B070EB36F070EB46F200EB56F2E
:10489000020EB66F010EB76FB86BB96BBA6BBB6B1C
:1048A000BC6BBD6BBE6BBF6BC06BC16BC26BC36BB4
:1048B000C46BC56BC66BC76BCA0E446F040E456FE5
:1048C000BB0E466F630E476F2A0E486F120E496F7C
:1048D000030E4A6F040E4B6FBB0E4C6F010E4D6FF3
:1048E0004E6B4F6B506B070E516F070E526F200EC1
:1048F000536F020E546F010E556F566B576B586B0A
:10490000596B5A6B5B6B5C6B5D6BB20E5E6F1D0E11
:104910005F6F000E606F000E616F626B636B646BA4
:10492000656BCA0E236F040E246F030E256F030EF2
:10493000266F120E276F120E286F030E296FC00EFE
:104940002A6F010E2B6F2C6B2D6B2E6B070E2F6FAA
:10495000070E306F200E316F020E326F010E336F73
:10496000346B356B366B376B386B396B3A6B3B6B33
:10497000EA0E3C6F1D0E3D6F000E3E6F000E3F6F46
:10498000406B416B426B436BCA0E0501C56F040E51
:10499000C66F1B0EC76F030EC86F120EC96F120EC3
:1049A000CA6F030ECB6F860ECC6F020ECD6FCE6B2F
:1049B000CF6BD06B070ED16F070ED26F200ED36F67
:1049C000020ED46F010ED56FD66BD76BD86BD96B37
:1049D000DA6BDB6BDC6BDD6B9E0EDE6F1D0EDF6F4B
:1049E000000EE06F000EE16FE26BE36BE46BE56BD2
:1049F000CA0EA46F040EA56F330EA66F030EA76F29
:104A0000120EA86F120EA96F030EAA6F880EAB6F5D
:104A1000020EAC6FAD6BAE6BAF6B070EB06F070ED7
:104A2000B16F200EB26F020EB36F010EB46FB56B93
:104A3000B66BB76BB86BB96BBA6BBB6BBC6B940ED8
:104A4000BD6F1D0EBE6F000EBF6F000EC06FC16B3D
:104A5000C26BC36BC46BCA0EE66F040EE76F4B0EDE
:104A6000E86F030EE96F120EEA6F120EEB6F030E82
:104A7000EC6F820EED6F020EEE6FEF6BF06BF16B71
:104A8000070EF26F070EF36F200EF46F020EF56F34
:104A9000010EF66FF76BF86BF96BFA6BFB6BFC6B47
:104AA000FD6BFE6B8A0EFF6F1D0E0601006F000E80
:104AB000016F000E026F036B046B056B066BCA0E71
:104AC000286F040E296F630E2A6F030E2B6F120ED0
:104AD0002C6F120E2D6F030E2E6F840E2F6F020E91
:104AE000306F316B326B336B070E346F070E356FDF
:104AF000200E366F020E376F010E386F396B3A6B2E
:104B00003B6B3C6B3D6B3E6B3F6B406BA80E416F4C
:104B10001D0E426F000E436F000E446F456B466BD7
:104B2000476B486BCA0E076F040E086F7B0E096F48
:104B3000030E0A6F120E0B6F120E0C6F030E0D6F29
:104B40008E0E0E6F020E0F6F106B116B126B070E35
:104B5000136F070E146F200E156F020E166F010EE5
:104B6000176F186B196B1A6B1B6B1C6B1D6B1E6B15
:104B70001F6BF40E206F1D0E216F000E226F000EB2
:104B8000236F246B256B266B276BCA0E0501836F81
:104B9000040E846F930E856F030E866F120E876F5F
:104BA000120E886F030E896F900E8A6F020E8B6F44
:104BB0008C6B8D6B8E6B070E8F6F070E906F200EB8
:104BC000916F020E926F010E936F946B956B966BC3
:104BD000976B986B996B9A6B9B6B1A0E9C6F1D0E63
:104BE0009D6F000E9E6F000E9F6FA06BA16BA26B5E
:104BF000A36BCA0E0401FF6F040E0501006FAB0E1C
:104C0000016F030E026F120E036F120E046F030E7C
:104C1000056F8A0E066F020E076F086B096B0A6B31
:104C2000070E0B6F070E0C6F200E0D6F020E0E6F2E
:104C3000010E0F6F106B116B126B136B146B156BF6
:104C4000166B176B100E186F1D0E196F000E1A6F72
:104C5000000E1B6F1C6B1D6B1E6B1F6BCA0E0401BD
:104C6000DE6F040EDF6FC30EE06F030EE16F120EF6
:104C7000E26F120EE36F030EE46F8C0EE56F020E0F
:104C8000E66FE76BE86BE96B070EEA6F070EEB6FF9
:104C9000200EEC6F020EED6F010EEE6FEF6BF06BFE
:104CA000F16BF26BF36BF46BF56BF66B5E0EF76FFB
:104CB0001D0EF86F000EF96F000EFA6FFB6BFC6BA8
:104CC000FD6BFE6BCA0E0501206F040E216FDB0E1B
:104CD000226F030E236F120E246F120E256F030E28
:104CE000266F800E276F020E286F296B2A6B2B6BA5
:104CF000070E2C6F070E2D6F200E2E6F020E2F6FDA
:104D0000010E306F316B326B336B346B356B366B3E
:104D1000376B386B800E396F1D0E3A6F000E3B6F8C
:104D2000000E3C6F3D6B3E6B3F6B406BCA0E626F7B
:104D3000040E636F0B0E646F1B0E656F120E666FB1
:104D4000120E676F030E686F740E696F020E6A6F42
:104D50006B6B6C6B6D6B070E6E6F070E6F6F200EBB
:104D6000706F020E716F010E726F736B746B756BE7
:104D7000766B776B786B796B7A6BEE0E7B6F240EAC
:104D80007C6F000E7D6F000E7E6F7F6B806B816B82
:104D9000826BCA0E416F040E426F230E436F1B0ECF
:104DA000446F120E456F120E466F030E476F760E5C
:104DB000486F020E496F4A6B4B6B4C6B070E4D6F81
:104DC000070E4E6F200E4F6F020E506F010E516F87
:104DD000526B536B546B556B566B576B586B596BCF
:104DE000680E5A6F1D0E5B6F000E5C6F000E5D6FDC
:104DF0005E6B5F6B606B616BCA0E0B018D6F040E97
:104E00008E6F3B0E8F6F1B0E906F120E916F120EF6
:104E1000926F030E936F700E946F020E956F966BE8
:104E2000976B986B070E996F070E9A6F200E9B6F0A
:104E3000020E9C6F010E9D6F9E6B9F6BA06BA16B12
:104E4000A26BA36BA46BA56BDA0EA66F230EA76FE4
:104E5000000EA86F000EA96FAA6BAB6BAC6BAD6BAD
:104E6000CA0E6C6F040E6D6F530E6E6F1B0E6F6F5C
:104E7000120E706F120E716F030E726F720E736FDF
:104E8000020E746F756B766B776B070E786F070E7B
:104E9000796F200E7A6F020E7B6F010E7C6F7D6B37
:104EA0007E6B7F6B806B816B826B836B846BE20E9E
:104EB000856F240E866F000E876F000E886F896BDA
:104EC0008A6B8B6B8C6BCA0EAE6F040EAF6F6B0E62
:104ED000B06F1B0EB16F120EB26F120EB36F030ED6
:104EE000B46F7C0EB56F020EB66FB76BB86BB96B53
:104EF000070EBA6F070EBB6F200EBC6F020EBD6FA0
:104F0000010EBE6FBF6BC06BC16BC26BC36BC46B5A
:104F1000C56BC66BB60EC76F230EC86F000EC96F88
:104F2000000ECA6FCB6BCC6BCD6BCE6BCA0EF06F25
:104F3000040EF16F830EF26F1B0EF36F120EF46FFF
:104F4000120EF56F030EF66F7E0EF76F020EF86FFE
:104F5000F96BFA6BFB6B070EFC6F070EFD6F200EF3
:104F6000FE6F020EFF6F010E0C01006F016B026BF2
:104F7000036B046B056B066B076B086BAA0E096F5E
:104F8000230E0A6F000E0B6F000E0C6F0D6B0E6B75
:104F90000F6B106BCA0E0B01CF6F040ED06F9B0E00
:104FA000D16F1B0ED26F120ED36F120ED46F030E81
:104FB000D56F780ED66F020ED76FD86BD96BDA6BC0
:104FC000070EDB6F070EDC6F200EDD6F020EDE6F4B
:104FD000010EDF6FE06BE16BE26BE36BE46BE56BA3
:104FE000E66BE76BFA0EE86F240EE96F000EEA6FCE
:104FF000000EEB6FEC6BED6BEE6BEF6BCA0E4B6F55
:10500000040E4C6FB30E4D6F1B0E4E6F120E4F6F92
:10501000120E506F030E516F7A0E526F020E536FC5
:10502000546B556B566B070E576F070E586F200E5B
:10503000596F020E5A6F010E5B6F5C6B5D6B5E6B9E
:105040005F6B606B616B626B636BFE0E646F1D0E5A
:10505000656F000E666F000E676F686B696B6A6B39
:105060006B6BCA0E0A01C76F040EC86FCB0EC96FF7
:105070001B0ECA6F120ECB6F120ECC6F030ECD6FCC
:10508000B50ECE6F000ECF6FD06BD16BD26B070E0B
:10509000D36F070ED46F200ED56F020ED66F010EA0
:1050A000D76FD86BD96BDA6BDB6BDC6BDD6BDE6BD0
:1050B000DF6BCE0EE06F230EE16F000EE26F000E8D
:1050C000E36FE46BE56BE66BE76BCA0EA66F040E4D
:1050D000A76F130EA86F330EA96F120EAA6F120ED0
:1050E000AB6F030EAC6FB70EAD6F000EAE6FAF6B54
:1050F000B06BB16B070EB26F070EB36F200EB46FBB
:10510000020EB56F010EB66FB76BB86BB96BBA6BA9
:10511000BB6BBC6BBD6BBE6BC20EBF6F230EC06F93
:10512000000EC16F000EC26FC36BC46BC56BC66B44
:10513000CA0EE86F040EE96F2B0EEA6F330EEB6FA9
:10514000120EEC6F120EED6F030EEE6FB10EEF6FDD
:10515000000EF06FF16BF26BF36B070EF46F070E3E
:10516000F56F200EF66F020EF76F010EF86FF96BF8
:10517000FA6BFB6BFC6BFD6BFE6BFF6B0B01006B4B
:10518000480E016F250E026F000E036F000E046FB4
:10519000056B066B076B086BCA0E2A6F040E2B6F2C
:1051A000430E2C6F330E2D6F120E2E6F120E2F6FBB
:1051B000030E306FB30E316F000E326F336B346BF2
:1051C000356B070E366F070E376F200E386F020EE5
:1051D000396F010E3A6F3B6B3C6B3D6B3E6B3F6B27
:1051E000406B416B426B3C0E436F250E446F000ECB
:1051F000456F000E466F476B486B496B4A6BCA0E92
:10520000096F040E0A6F5B0E0B6F330E0C6F120EDC
:105210000D6F120E0E6F030E0F6FBD0E106F000E8E
:10522000116F126B136B146B070E156F070E166F51
:10523000200E176F020E186F010E196F1A6B1B6B81
:105240001C6B1D6B1E6B1F6B206B216B600E226F26
:10525000250E236F000E246F000E256F266B276B23
:10526000286B296BCA0E0C01116F040E126F730E9E
:10527000136F330E146F120E156F120E166F030E8E
:10528000176FBF0E186F000E196F1A6B1B6B1C6B1C
:10529000070E1D6F070E1E6F200E1F6F020E206F70
:1052A000010E216F226B236B246B256B266B276B02
:1052B000286B296B540E2A6F250E2B6F000E2C6F56
:1052C000000E2D6F2E6B2F6B306B316BCA0EB06FD3
:1052D000040EB16F8B0EB26F330EB36F120EB46F3C
:1052E000120EB56F030EB66FB90EB76F000EB86F22
:1052F000B96BBA6BBB6B070EBC6F070EBD6F200E90
:10530000BE6F020EBF6F010EC06FC16BC26BC36B6D
:10531000C46BC56BC66BC76BC86B120EC96F250E0D
:10532000CA6F000ECB6F000ECC6FCD6BCE6BCF6B08
:10533000D06BCA0E8F6F040E906FA30E916F330E59
:10534000926F120E936F120E946F030E956FBB0E39
:10535000966F000E976F986B996B9A6B070E9B6F09
:10536000070E9C6F200E9D6F020E9E6F010E9F6FA9
:10537000A06BA16BA26BA36BA46BA56BA66BA76BB9
:10538000060EA86F250EA96F000EAA6F000EAB6F58
:10539000AC6BAD6BAE6BAF6BCA0ED16F040ED26F40
:1053A000BA0ED36F330ED46F320ED56F120ED66F86
:1053B000320ED76F120ED86F7A0ED96F620EDA6F77
:1053C000000EDB6F010EDC6FDD6BDE6BDF6BE06B05
:1053D000E16BE26BE36BE46BE56B2A0EE66F250E87
:1053E000E76F000EE86F000EE96FEA6BEB6BEC6B9A
:1053F000ED6BCA0E0D010E6F040E0F6F1B0E106FBA
:105400004B0E116F720E126F120E136F030E146F8C
:10541000A30E156F000E166F176B186B196B070E26
:105420001A6F070E1B6F200E1C6F020E1D6F010EF0
:105430001E6F1F6B206B216B226B236B246B256B04
:10544000266B1E0E276F250E286F000E296F000E8B
:105450002A6F2B6B2C6B2D6B2E6BCA0E0C01EE6F13
:10546000040EEF6F080EF06F680EF16F010EF26F11
:10547000080EF36F200EF46F000EF56FF66BF76BEE
:10548000F86B070EF96F070EFA6F200EFB6F020E16
:10549000FC6F010EFD6FFE6BFF6B0D01006B016B6E
:1054A000026B036B046B056B066B076B086B096B78
:1054B0000A6B0B6B0C6B0D6BCA0E0C01546F040E58
:1054C000556F050E566F630E576FB00E586F130E63
:1054D000596F010E5A6F5B6B5C6B5D6B5E6B5F6B44
:1054E000606B616B626B636B646B656B666B676B48
:1054F000686B696B6A6BCA0E326F040E336F9B0E5A
:10550000346F4B0E356F520E366F120E376F030E1F
:10551000386F040E396F350E3A6F000E3B6F3C6BDF
:105520003D6B3E6B070E3F6F070E406F200E416FC5
:10553000020E426F010E436F446B456B466B476B27
:10554000486B496B4A6B4B6BC00E4C6F1F0E4D6F17
:10555000000E4E6F000E4F6F506B516B526B536BC2
:105560006B0E0801C26F0C0EC36FBB0EC46F630ECF
:10557000C56F2A0EC66F120EC76F030EC86F040EDA
:10558000C96F150ECA6F000ECB6FCC6BCD6BCE6B97
:10559000070ECF6F070ED06F200ED16F020ED26FA5
:1055A000010ED36FD46BD56BD66BD76BD86BD96B21
:1055B000DA6BDB6BB20EDC6F1F0EDD6F000EDE6F81
:1055C000000EDF6FE06BE16BE26BE36B6B0EA26FC3
:1055D0000C0EA36F600EA46F100EA56F280EA66FA1
:1055E000080EA76F1A0EA86F000EA96FAA6BAB6BFF
:1055F000AC6B070EAD6F070EAE6F200EAF6F020ED5
:10560000B06F010EB16FB26BB36BB46BB56BB66BB1
:10561000B76BB86BB96BBA6BBB6BBC6BBD6BBE6B5E
:10562000BF6BC06BC16B6B0EE46F0C0EE56F080EA9
:10563000E66F200EE76FB80EE86F080EE96F700E88
:10564000EA6F000EEB6FEC6BED6BEE6B070EEF6F1E
:10565000070EF06F200EF16F020EF26F010EF36F66
:10566000F46BF56BF66BF76BF86BF96BFA6BFB6B26
:10567000FC6BFD6BFE6BFF6B0901006B016B026B3A
:10568000036B6B0E246F0C0E256F080E266F280E11
:10569000276FD00E286F080E296F880E2A6F000E14
:1056A0002B6F2C6B2D6B2E6B070E2F6F070E306F31
:1056B000200E316F020E326F010E336F346B356B7B
:1056C000366B376B386B396B3A6B3B6B3C6B3D6BB6
:1056D0003E6B3F6B406B416B426B436B6B0E046FD9
:1056E0000C0E056F080E066F300E076FC00E086FA8
:1056F000080E096F3F0E0A6F000E0B6F0C6B0D6BDF
:105700000E6B070E0F6F070E106F200E116F020E3B
:10571000126F010E136F146B156B166B176B186BF2
:10572000196B1A6B1B6B1C6B1D6B1E6B1F6B206B3D
:10573000216B226B236B6B0E0801826F0C0E836F43
:10574000080E846F380E856FB80E866F080E876F4F
:10575000580E886F000E896F8A6B8B6B8C6B070EEF
:105760008D6F070E8E6F200E8F6F020E906F010EE1
:10577000916F926B936B946B956B966B976B986B29
:10578000996B9A6B9B6B9C6B9D6B9E6B9F6BA06BDD
:10579000A16B6B0E3A6F0C0E3B6F080E3C6F400E08
:1057A0003D6FE00E3E6F080E3F6F040E406F010E1E
:1057B000416F426B436B446B070E456F070E466F9C
:1057C000200E476F020E486F010E496F4A6B4B6BFC
:1057D0004C6B4D6B4E6B4F6B506B516B526B536BF5
:1057E000546B556B566B576B586B596B6B0E1A6F2E
:1057F0000C0E1B6F080E1C6F480E1D6FD00E1E6F17
:10580000080E1F6F210E206F010E216F226B236B7C
:10581000246B070E256F070E266F200E276F020ED2
:10582000286F010E296F2A6B2B6B2C6B2D6B2E6B47
:105830002F6B306B316B326B336B346B356B366B7C
:10584000376B386B396B5A0E0A01206F080E216FC7
:10585000BB0E226F630E236F2A0E246F120E256F6C
:10586000030E266F040E276FF90E286F000E296FA6
:105870002A6B2B6B2C6B070E2D6F070E2E6F200ED5
:105880002F6F020E306F010E316F326B336B346B42
:10589000356B366B376B386B396B4A0E3A6F200EAF
:1058A0003B6F000E3C6F000E3D6F3E6B3F6B406BDD
:1058B000416B5A0E0901FE6F080EFF6F130E0A01AD
:1058C000006F0B0E016F320E026F120E036F030E8C
:1058D000046F040E056FFE0E066F000E076F086B57
:1058E000096B0A6B070E0B6F070E0C6F200E0D6F06
:1058F000020E0E6F010E0F6F106B116B126B136B9C
:10590000146B156B166B176B080E186F200E196F42
:10591000000E1A6F000E1B6F1C6B1D6B1E6B1F6B36
:105920005A0E426F080E436F5B0E446F0B0E456FAD
:10593000320E466F120E476F030E486F040E496F0A
:10594000440E4A6F010E4B6F4C6B4D6B4E6B070E46
:105950004F6F070E506F200E516F020E526F010EE7
:10596000536F546B556B566B576B586B596B5A6B27
:105970005B6B4A0E5C6F1E0E5D6F000E5E6F000E5D
:105980005F6F606B616B626B636B5A0E846F080EA6
:10599000856FA30E866F0B0E876F320E886F120E07
:1059A000896F030E8A6F040E8B6F4A0E8C6F010E87
:1059B0008D6F8E6B8F6B906B070E916F070E926FD2
:1059C000200E936F020E946F010E956F966B976B7E
:1059D000986B996B9A6B9B6B9C6B9D6B080E9E6F83
:1059E0001E0E9F6F000EA06F000EA16FA26BA36B27
:1059F000A46BA56B5A0E646F080E656F200E666F60
:105A0000200E676F100E686F080E696F3C0E6A6F8C
:105A1000010E6B6F6C6B6D6B6E6B070E6F6F070E0D
:105A2000706F200E716F020E726F010E736F746BC8
:105A3000756B766B776B786B796B7A6B7B6B7C6B4A
:105A40007D6B7E6B7F6B806B816B826B836B5A0E81
:105A50000901DE6F080EDF6F680EE06F200EE16F48
:105A6000100EE26F080EE36F400EE46F010EE56F5B
:105A7000E66BE76BE86B070EE96F070EEA6F200E27
:105A8000EB6F020EEC6F010EED6FEE6BEF6BF06BD8
:105A9000F16BF26BF36BF46BF56BF66BF76BF86B0A
:105AA000F96BFA6BFB6BFC6BFD6B5A0E666F080EA5
:105AB000676FB00E686F200E696F100E6A6F080E68
:105AC0006B6FF50E6C6F000E6D6F6E6B6F6B706BA6
:105AD000070E716F070E726F200E736F020E746FD8
:105AE000010E756F766B776B786B796B7A6B7B6B6E
:105AF0007C6B7D6B7E6B7F6B806B816B826B836B52
:105B0000846B856B5A0E446F080E456F3B0E466FD3
:105B1000330E476F720E486F120E496F030E4A6FB5
:105B2000040E4B6FD90E4C6F000E4D6F4E6B4F6BCA
:105B3000506B070E516F070E526F200E536F020EFF
:105B4000546F010E556F566B576B586B596B5A6BF0
:105B50005B6B5C6B5D6B4A0E5E6F1F0E5F6F000EC2
:105B6000606F000E616F626B636B646B656B5A0EE6
:105B7000866F080E876F3B0E886F4B0E896F720E13
:105B80008A6F120E8B6F030E8C6F040E8D6FE70EF3
:105B90008E6F000E8F6F906B916B926B070E936FF1
:105BA000070E946F200E956F020E966F010E976F81
:105BB000986B996B9A6B9B6B9C6B9D6B9E6B9F6BB1
:105BC0008C0EA06F1E0EA16F000EA26F000EA36FB1
:105BD000A46BA56BA66BA76B5A0EBC6F080EBD6FAE
:105BE0003B0EBE6F630EBF6F720EC06F120EC16FA1
:105BF000030EC26F040EC36FC10EC46F000EC56FDB
:105C0000C66BC76BC86B070EC96F070ECA6F200E35
:105C1000CB6F020ECC6F010ECD6FCE6BCF6BD06B06
:105C2000D16BD26BD36BD46BD56B580ED66F200E65
:105C3000D76F000ED86F000ED96FDA6BDB6BDC6BA1
:105C4000DD6BA80E03019E6F090E9F6F9B0EA06F68
:105C50006B0EA16F520EA26F120EA36F030EA46FF4
:105C6000CF0EA56F000EA66FA76BA86BA96B070ED2
:105C7000AA6F070EAB6F200EAC6F020EAD6FAE6B4E
:105C8000AF6BB06BB16BB26BB36BB46BB56BB66B28
:105C9000280EB76F210EB86F000EB96F000EBA6FE5
:105CA000BB6BBC6BBD6BBE6B12000900F5CFE6FF92
:105CB0000006FBE10106F9E1120093EC17F0300E4B
:105CC0000D012F6F000E306FB30E316F030E326F68
:105CD000580E336F000E346F820E356F030E366F21
:105CE000B9EC1EF0F1EC1FF0DF0E0D01476F060E50
:105CF000486F26EC0EF01200CAEC1EF0005228E0AD
:105D00009A0E2F6F030E306F9C0E316F030E326FA1
:105D100004EC1FF00050000A1AE19AC32FFD9BC348
:105D200030FD9CC331FD9DC332FDC0EC14F0030176
:105D30009751000A0CE1010E976F9AC32FFD9BC388
:105D400030FD9CC331FD9DC332FDCDEC1BF00FD067
:105D500003019751010A0BE1976B9AC32FFD9BC377
:105D600030FD9CC331FD9DC332FDDAEC17F012000B
:105D700012007CEC31F0A1DFBFDFFED7FFD74E650C
:105D8000787400494E464F3A0000000000000000C1
:105D9000000000000000000000000000000043417F
:105DA00050533A204F464600636F6D706F6E656EBC
:105DB0007473206F66206261636B6C696768742E10
:105DC00000436F6D706C657465207475726E204F42
:105DD0004E2F4F4646206F66004261636B6C6967C9
:105DE00068742044656D6F206C65747320796F75DD
:105DF000006368616E6765205265642C20426C7593
:105E00006520616E6420477265656E002020202049
:105E100053706163652020202000580043004C002F
:105E20005A004E004D00560042004261636B6C699F
:105E3000676874204F4646004D61696E206D656E3F
:105E400075004261636B6C69676874204F4E200077
:105E500020496E76657274205247422020004F4ED2
:105E600000004261636B00205245442000617320B2
:105E700077656C6C20617320696E76657274696EEB
:105E800067206F6620656163680052474220636F38
:105E90006D706F6E656E7420696E64697669647585
:105EA000616C792E004F4E00004F4E0000424C5561
:105EB000452000475245454E004261636B73706157
:105EC00063652066756E6374696F6E7320617265B9
:105ED00020616C736F00737570706F727465642EDF
:105EE00020546F2072657475726E20746F206D611E
:105EF000696E00697320646973706C6179656420F0
:105F0000696E20626F74746F6D206261722E00532F
:105F1000706163652C2043617073204C6F636B204C
:105F2000616E64004261636B00510073637265656A
:105F30006E207072657373204261636B2E00494E50
:105F4000464F3A006B6579626F6172642E2045613D
:105F50006368206B65792070726573736564006295
:105F600079204D696B726F456C656B74726F6E69E9
:105F70006B610020204B65797061642044656D6F12
:105F800020202000536D61727420474C434420321E
:105F9000343078313238004E657874004B65797052
:105FA00061642044656D6F2073686F7773206F6E36
:105FB00073637265656E004261636B6C69676874D8
:105FC000204368616E6765004261636B6C69676856
:105FD0007420436F6C6F727300440046004100539D
:105FE000004A004B00470048005000520054005740
:105FF00000450049004F00590055002020475245F8
:10600000454E2020202020002020524544202020E2
:1060100020202020004F4E20002020574849544582
:10602000202020002059454C4C4F57202020200094
:1060300054555251554F49534520202020200020CF
:1060400020424C554520202020004F4E20004F4E2E
:1060500020004F4646004F4E20004F4646004F4E10
:1060600020004F4E20004F4E20004F46460000209B
:10607000505552504C4520202020000000000000C8
:106080000000000000000000000000000000000010
:10609000004F4646004F4E2000434150533A2020C7
:1060A0004F4E00434150533A204F4646004F46461C
:1060B000004F4646004F4646004F4646004F4E2092
:1060C00000202020202020202020202020202020F0
:1060D00020202020202020000000434150533A205F
:1060E0004F4646004F4646002020202020202020FA
:1060F00020202020202020202020202020200000E0
:106100003FFFFFFFFFFFF07FFFFFFFFFFFFCE0000F
:10611000000000000CDFFFFFFFFFFFF6DFFFFFFFC7
:10612000FFFFF6DF01FFF007FFF6DC007F8000FFD6
:10613000F6DC003E00003FF6DCFF3C00000FF6DD21
:10614000FF30000007F6DC0070000007F6DC00609E
:10615000000003F6DE00E001C001F6DFFFC001E051
:1061600001F6DFFFC003E001F6DC7FC003E000F6CC
:10617000DC3FC003E000F6DC01C003E000F6DC0118
:10618000C003E000F6DC01C003E000F6DFFFC00161
:10619000E000F6DDFDC0000000F6DC31C0000000CC
:1061A000F6DC21C0000000F6DF03C0000000F6DDD1
:1061B00001C0000000F6DC01C0000000F6DC01C0F8
:1061C00001FFFFF6DDFFC003FFFFF6DFFFC003FFA7
:1061D000FFF6DD81C003F000F6DD81C003F000F6BC
:1061E000DD01C003F000F6DFFFC003F000F6DFFFC3
:1061F000C003F000F6DC01C003F000F6DC01C003D0
:10620000F000F6DC00C003F000F6DDFFC003F00094
:10621000F6DFFFC001E001F6DC00E001E001F6DCA2
:106220000060008001F6DC0070000003F6DDFFF086
:10623000000007F6DDFFF800000FF6DC001C000090
:106240001FF6DC000F00003FF6DC0007C000FFF681
:10625000DFFFFFFFFFFFF6DFFFFFFFFFFFF6DFFFC0
:10626000FFFFFFFFEE6000000000000C7FFFFFFF5C
:10627000FFFFF81FFFFFFFFFFFF0FFE1FFFFFFFF42
:10628000C0FFC1FFFFFFFFC0FF81FFFFFFFFC0FF97
:1062900003FFFFFFFFC0FE07FFFFFFFFC0FC0FFF74
:1062A000FFFFFFC0FC00000000FFC0F8000000007E
:1062B000FFC0F800000000FFC0FC00000000FFC0AD
:1062C000FC00000000FFC0FE0FFFFFFFFFC0FF0744
:1062D000FFFFFFFFC0FF03FFFFFFFFC0FF81FFFFC6
:1062E000FFFFC0FFC1FFFFFFFFC0FFC1FFFFFFFFB8
:1062F000C0FFE3FFFFFFFFC010EE15F0820E006E3F
:10630000040E016E7E0EF66E5D0EF76E000EF86ED8
:1063100055EC2EF01200FFFFFFFFFFFFFFFFFFFF16
:10632000FFFFFFFFFFFFFFFFFFFFFFFFFFFFFFFF7D
:10633000FFFFFFFFFFFFFFFFFFFFFFFFFFFFFFFF6D
:10634000FFFFFFFFFFFFFFFFFFFFFFFFFFFFFFFF5D
:10635000FFFFFFFFFFFFFFFFFFFFFFFFFFFFFFFF4D
:10BD0000FFFFFFFFFFFFFFFF070EAF6EAC8479D888
:10BD1000670E5D6E720E5E6EA0D8005202E0B4D85F
:10BD200001D04ED9FFD7F2CF01F06DC0F6FF6EC043
:10BD3000F7FF6FC0F8FFA68EA69CA684A688F29E89
:10BD4000550EA76EAA0EA76EA682F28E0A0071C0CB
:10BD5000E9FF72C0EAFF036A010E035C14E2026AA3
:10BD6000400E025C05E2EECFF5FF0F00022AF8D785
:10BD7000A68EA69CA684F29E550EA76EAA0EA76E4E
:10BD8000A682032AE9D7F28EA69401C0F2FF120020
:10BD9000ACB202D00000FCD760C0ADFF1200C00EF4
:10BDA00000016D6FBF0E6E6F000E6F6F706F1D0E16
:10BDB000716F000E726FB7DF840E1D6EEF0E1E6E78
:10BDC0005E0E1F6EF00E206E1200000E9EBA010E67
:10BDD000016E01C000F01200AECF02F0ABA202D0A3
:10BDE000AB98AB8802C001F001C000F01200540E05
:10BDF0000C6E1C0E0D6E0D2EFED70C2EFCD7000007
:10BE00001200900E196EBD0E1A6E600E1B6E000EA3
:10BE10001C6ED80E156EBD0E166E000E176E000E3F
:10BE2000186ECA0E0001656FBD0E666F000E676F5B
:10BE3000000E686FFF0E616FFF0E626F000E636F82
:10BE4000000E646FAC8A900EAB6E948E949C9EAA8A
:10BE500003D0AECF00F0FBD712005F6AC8DF5DC031
:10BE600060F096DFC4DF5F2A5F50FF0A02E15F6A7D
:10BE700008D0B2DF00505E1803E1010E5F6E01D002
:10BE8000EDD75FC000F012005D6A0001696B6A6B5C
:10BE90006B6B6C6B5D50400A25E10001000E006E7B
:10BEA0006C1908E100506B1905E100506A1902E1B4
:10BEB0006951000A01E173DF69C06DF06AC06EF07C
:10BEC0006BC06FF06CC070F01D0E0001716F000E42
:10BED000726F29DF5D6A400E00016927000E6A2338
:10BEE0006B236C230001790E606F52DF6EDF005010
:10BEF000000AFCE071DF00C05FF0780E0001606FA7
:10BF000047DF63DF0050000AFCE066DF00C05EF040
:10BF10001D0EE16E000EE26E5D50E126D8B0E22A01
:10BF20005FC0E6FF5D2A1D0EE16E000EE26E5D5001
:10BF3000E126D8B0E22A5EC0E6FF5D2AABD7120048
:10BF4000FFFFFFFFFFFFFFFFFFFFFFFFFFFFFFFF01
:10BF5000FFFFFFFFFFFFFFFFFFFFFFFFFFFFFFFFF1
:10BF6000FFFFFFFFFFFFFFFFFFFFFFFFFFFFFFFFE1
:10BF7000FFFFFFFFFFFFFFFFFFFFFFFFFFFFFFFFD1
:10BF8000FFFFFFFFFFFFFFFFFFFFFFFFFFFFFFFFC1
:10BF9000FFFFFFFFFFFFFFFFFFFFFFFFFFFFFFFFB1
:10BFA000FFFFFFFFFFFFFFFFFFFFFFFFFFFFFFFFA1
:10BFB000FFFFFFFFFFFFFFFFFFFFFFFFFFFFFFFF91
:10BFC000B9EF2EF00000000000EF00F000000000CC
:10BFD0000000000000000000F3D7FFFF020E0D6E0E
:10BFE0000D2EFED7000012008880FF0E996E8892F9
:10BFF000030E8714016E0150030A01E0F9D788820D
:0200000400F00A
:08000000FFFFFFFFFFFFFFFF00
:08000800FFFFFFFFFFFFFFFFF8
:08001000FFFFFFFFFFFFFFFFF0
:08001800FFFFFFFFFFFFFFFFE8
:020000040020DA
:020000040030CA
:0E0000000006011EF383800007C007E00740E2
:00000001FF
